:020000041100E9
:10300000002373B52B4D2C4C28006361022601F080
:1030100081F94021FE2221742800284B009601F0FE
:10302000CBF9002836D1217CFF222800244B0096C2
:1030300001F0C2F900282DD1224BA2899A4226D153
:10304000E389214A93420DD1204B6361204B2268D2
:10305000002A03D1002B01D043CB43C4280001F048
:1030600097F973BD1B4A934201D00023EFE71A4B37
:103070001A4A1B68934206D9C02304222800217CE7
:103080009B0001F00FFA114B6361154BDFE7002342
:103090002374EAE7CC233821AC2228009B01217459
:1030A00001F000FA0028F2D10E4B63610E4BE38170
:1030B0000E4BCCE7F441FF1F9061FF1F9C61FF1F87
:1030C0009E61FF1F59590000830500004141001116
:1030D00068B9001182150000B461FF1F871300005A
:1030E00074B90011F9410011AAAAFFFF5CB90011DF
:1030F000F7B5164B0192C318021D002000938823D8
:103100005B05D3181B685C1C1AD09CB2402C18D8E5
:103110008D781E0CAC466746CD782D023D43AE42FD
:1031200006D1019800280ED110000C70240A4C70B2
:1031300003249BB20733A343D218009B9A42DED3E9
:10314000FEBD4432F9E71000FAE7C046FC0F00006C
:10315000802213B503000324019189B25201073183
:103160009B18A14304305A1A88235B05C3181B68B7
:10317000591C03D190429241104016BD99B240298A
:1031800007D80B000733A343C0189042ECD30020AC
:10319000F3E74430F9E7134B134A1B68126810B584
:1031A000FA24934201D81A00F824104BE4021B6859
:1031B0009A4210D813000E4A12689A420ED3013375
:1031C00007D1F823DB029C4203D10A49054808F0E5
:1031D0003FFB200010BDFC24E402ECE7FE24E402E7
:1031E000F7E7C04600C0071100D0071100E0071143
:1031F00000F00711FFFFFF7FF0B59BB015000490B2
:103200000391402A00D9A0E006AB59801A80FFF74D
:10321000C2FF0400042816D9002206A9FFF768FFA0
:10322000052810D906AB1B88AB420CD1002D07D066
:10323000514B2A000499C01808F00AFA002802D15C
:1032400001201BB0F0BD06AB1D8020000699FFF7E2
:103250007FFF041E7BD1069B0793FFF79CFF802313
:103260005B01C618802307001B039E4201D3F8268A
:10327000F60288235B05F31801931B68013302D023
:10328000019808F0EDF83D49019808F0E1FA3B1D7E
:103290000293331D05938822029B52059B181B68DD
:1032A00008935A1C3CD044219AB20091402A04D879
:1032B0000320D11D814389B2009103991B0C8B42DD
:1032C00024D0402A22D80122300008A9FFF710FF9D
:1032D000021E1BD1380008A9FFF70AFF04000428CA
:1032E00031D9009A059B9B1880225201B218934253
:1032F00040D288235B05C118009A09A808F008FA93
:103300001D4B009A09A9F01808F082FA009A029B56
:103310009446634402931A4B029AFB189A42BAD31A
:1033200088235B05FC1821680198013908F090FAA0
:10333000200008F095F8039A07AB5A8030000799EF
:10334000FFF706FF0400002C03D1002079E70428D2
:10335000FBD988235B05E018069908F079FA032366
:10336000EA1C9A4300D16BE7034B0499E01808F07C
:103370004FFA65E70424ECE704000011FFFFFF7F2C
:10338000F80F0000F7B505001400402A21D80027E7
:1033900001AE71803780FFF7FEFE042816D93A008F
:1033A0003100FFF7A5FE042810D93688BC420BD0A7
:1033B000BD4209D0221CB44200D9321C064B92B245
:1033C000C118280008F0A4F930B2FEBDC04300B215
:1033D000FBE703204042F8E70400001137B5042260
:1033E00004000D0001A81649FFF7CCFF02000428D5
:1033F0000BD1019BA34208D3AB4204D0104901A8D2
:103400000195FFF7F9FE01203EBD0E4C2368200018
:10341000019308F025F8019920000139019108F085
:1034200017FA80235B01E418074B9C42EED104227B
:10343000034901A80195FFF7DFFE0020E4E7C0463D
:103440005555000000C007110000081130B589B0C3
:1034500008F03EF810226946254807F071FF254B19
:10346000009A9A420ED1019B029A0F2B33D8002169
:1034700001240698013B08D2002900D00292029B49
:10348000013331D10023029325E0551CF2D1020013
:103490002100EFE710341022200004A907F050FFAC
:1034A000029B013301D1069B0293882304995B059B
:1034B000C918059B06981A03120B049105928142C4
:1034C00003D02B4201D108F023F9019B013B01936A
:1034D000019B002BDED1029B002B03D004930498A8
:1034E0004168084709B030BDE025014C2D03EFE7E6
:1034F00000000111504859368022F8B5964C974B80
:10350000D200002120001C6007F0C2FF2300944A73
:1035100088331A60934B1A786A23002A00D011333B
:10352000E3620A232365904B37221B780820A363AC
:103530008E4B2118E361102323628D4B3B25636181
:10354000C823DB00A36123008C331A602823013ACF
:10355000E26320646364CA67043A211DCA672100DC
:10356000BC310D602100C03108602100C4310B6006
:1035700021000635CC310D602100083DC8310D60B9
:103580002100D0310A602200D43210602200D832EB
:10359000136022000227E032210017604222DC3152
:1035A0000A6021001B3DE4310D602100E831086014
:1035B0002100EC310B6023000521F4331960230056
:1035C000F0331A602300183290331A6023009433CA
:1035D000186023001E3A98331A60AF23DB00236083
:1035E000644BFA262363644B644DE360644BF03113
:1035F000A3642300FF31FC33B600A16021611E608B
:10360000A5627325E5656D3D6565A56596255D4AF1
:10361000AD00E264666258606766A566002709250A
:10362000A767E566584F594D606720002567E26738
:103630003A6015279C30676007001A203860200028
:10364000A0300700212038602000A83007004C4837
:1036500038602000F830066026006427A436376002
:1036600026005F3FAC3637602600033FB036376038
:103670002600C637B436376026000027B8363760D4
:1036800038269E60424E96205E64424E5A66DE6147
:10369000414E9A645E62F53EFF3E9E621E269A6728
:1036A000354A8000DE661F675F67DD651D6618624C
:1036B000DA67BE23394A5B00E250394BD8382350D1
:1036C00004302250C4225200A350C623E4205B00E1
:1036D000E1500433334AE1503349344BD16034492B
:1036E000800019503349E938FF3819503249043005
:1036F000195032493248D16132491163324951631C
:103700001900F4310860CE20304940001160304982
:10371000195019002F48F83108602F49D1658221CE
:103720002E4A89005A501A002D490832D1671A00D2
:103730002C49B432116088212B4A89005A501A0052
:103740002A49883211602A4ADA6407F0F9FE01201A
:1037500007F0A6FDF8BDC0460004FF1F2C64FF1F44
:10376000106FFF1F2444FF1F4A0AFF1F3A07000083
:1037700080C3C9019A020000DC0500006A1800003D
:1037800050C3000088130000F009FF1F204E000006
:103790006509FF1F68100000C409000040420F00C7
:1037A00010270000FC00FF1FC11BFF1F0000FF1FB0
:1037B000152CFF1FA52FFF1F3D2EFF1F811FFF1F71
:1037C0007126FF1F9D1FFF1F4921FF1F0D1FFF1F98
:1037D0009528FF1F7D29FF1FD918FF1FA127FF1F55
:1037E000C524FF1FD124FF1F0D1EFF1FC51EFF1F75
:1037F000851DFF1F0223F0B50124634D634E2B701E
:10380000634B91B01C70634F039333680021082011
:10381000BB7006F009FC082006F000FB002398426C
:1038200005D0BA78552A02D0332A00D09FE0336001
:10383000042006F073FD07F003FEFFF75DFE07F0BE
:103840004FFD1F2201240021534B10AE1A70534B21
:103850001C70534B1970534B19689143163A0A4325
:103860001A60602219689143403A0A431A6007F0CF
:10387000EFFC07F01DFDC120FF214B4B80001A58C3
:103880008A431A50C522920098588843BF39014391
:1038900099509858454908408021C901014380202A
:1038A00099509958C0050902090A0143995080218D
:1038B0003F48490107F094FE032322003D4901944B
:1038C00000933D4807F00CFF2C223C4905A807F067
:1038D0001FFF05AC61782078023406F0BFFAA642DB
:1038E000F8D1374C0121002006F0CCFB0920012142
:1038F00006F0C8FB2268334B03201A40A023DB02EA
:1039000013432360802322689B04134323602268AF
:103910002D4B1A4080239B03134323602B4A2C4BCF
:10392000934200D8012007F023FD07F099FE802381
:103930002268DB0413432360287807F021FF039BF0
:103940001878C0B207F044FE07F0F2FE21490420C7
:1039500007F02EFE06F0AEFC00F0A8F800F0CEFD59
:1039600000F076FE00F01AFA002011B0F0BD0093CE
:103970002100184A042007F0DBFD8023DB059C6250
:10398000FFF764FD54E7C0464A0AFF1F34F00040C9
:103990002444FF1FC061FF1F480AFF1F490AFF1F81
:1039A000680AFF1FBCF0004000E100E0FF00FFFFDD
:1039B0002844FF1FAC56FF1F2854FF1F80B800117A
:1039C00014F00040FF7FF8FFFFFF9FFF0080FF1F04
:1039D000106FFF1F3B00010870B500252549264ADE
:1039E00026484D6308CA1B051B0DED188242F9D10C
:1039F00000268022224B92058B630921214B224C09
:103A00001E62224B1120DA67214BDA688A43DA60A2
:103A10009A6820490A409A60266007F011FF112039
:103A200007F02EFD8022636C93436364EE24E40070
:103A30006C43194A200C0400642390420AD8FA22ED
:103A40003300D200904205D9144B0A21C01807F068
:103A5000B7FCC3B2124A11201372D48007F020FDC4
:103A6000104B1B78002B04D10F4B1021187807F056
:103A7000FFFD70BD000005408805054000060540BB
:103A8000FF01000000F000400038004004E100E0C9
:103A90003CF00040FFDFFFFFB70B000030F8FFFFF6
:103AA000A861FF1FE263FF1FE061FF1F002210B546
:103AB0001100112007F0B4FC10BD0000F8B5002380
:103AC0000926374F374C3B62E3681120B343E3606C
:103AD00007F0D6FC112007F0B3FE112007F0D8FB49
:103AE0004023226880251343236080236268DB0221
:103AF00013436360A3682C4A2B43A360A36802218D
:103B00001340A3608023A2689B0113431022A3608B
:103B1000236C072093432364236C0F3A13432364DD
:103B200080235B003B62226B204B1A402263626B56
:103B30001A406263A26B1A40A263E26B1340E36314
:103B4000E3681B4A1340E36006F088F9012107206F
:103B500006F098FA174B11205A6C15435D6407F074
:103B600017FCFD21144B154A89005A508023C720A9
:103B7000626B5B0313436363E36880003343E3607A
:103B80000F4B104A19581140802212020A431A5052
:103B9000802292051A6008220B4B5A63F8BDC0467A
:103BA00000F000403CF00040FFFFDFFFEFFFEFFFC1
:103BB000FFFF7FFF003800400000FF1FD9390011D0
:103BC00000E100E0FF00FFFF0000054030B503A862
:103BD00004880B20002C0ED14968074D08784978DD
:103BE000090201430A20A94205D1012120001980C0
:103BF000024B1B7A137030BD192A0000A861FF1F09
:103C0000F7B5150008AA16884A680F4F147852783D
:103C1000120222430A24BA4214D10122DBB20192D9
:103C200000962A0007F096FA041E0BD1074B1B687A
:103C3000002B07D068782A78000210434242504196
:103C4000013098472000FEBD022900002C61FF1FB3
:103C500030B5012503790400BFB02B4211D00A49C9
:103C6000408806F0E3FD28420BD0084B01A95B8D8C
:103C70004D800B80064B00221B7A60880B7103F08D
:103C8000B5FE3FB030BDC0462461FF1F6840FF1F36
:103C9000A861FF1F10B50549054806F07DFD042108
:103CA000044A054806F03AFD10BDC0462461FF1FD6
:103CB000FFFF0000ACB800116840FF1F10B50248BC
:103CC00004F016FD10BDC046513C001101230370E5
:103CD0000B4B1A7A4270022282709A78C270DA789C
:103CE0000271032242711A7982715A79C2710C22CF
:103CF00002729A794272DB7983720B207047C04658
:103D0000A861FF1F022310B50370013B4370053308
:103D1000837010330371443B43712A3383714433FE
:103D2000C37100230372064B04001B8843720A30E0
:103D3000FFF7CCFF831D0A30C0B2E37010BDC04650
:103D4000A861FF1F10B5142007F01AFC124B1422B3
:103D50000021186007F09CFB002007F001FC012007
:103D600007F0F6FB022007F0CBFB032003F064FF13
:103D7000042005F079FF052003F0A2F9062003F0E6
:103D80006FFE072001F006FA082006F0A7FC0920C4
:103D900000F0E8FF10BDC0463061FF1F07F030FCA7
:103DA000012007F025FB07F093FC0000094B10B53C
:103DB0000400984205D0012904D12000064906F0EC
:103DC000EBFC10BD0229FCD1013904F04FFC0028A6
:103DD000F3D0F6E7FEFF00005661FF1F70B50D7AC5
:103DE000100004AA2C00168810221440154220D17D
:103DF000002E20D10A78022A18D14A685178157805
:103E00000E4A09022943914205D00D4A914209D038
:103E10001C800A2404E014220A491A8007F078FC66
:103E2000200070BD0C2208491A80F7E71C8001248D
:103E3000F6E70824F4E70B24F2E7C046F3FF00009E
:103E4000F4FF0000B042FF1F8CB9001110B5040050
:103E50000749084806F0A0FC074804F089FB002049
:103E6000E40704D50721054A054806F057FC10BDB4
:103E70005661FF1FFFFF0000AD3D0011F0B80011BB
:103E8000AC40FF1F00B50C4BBFB01A780B4902A81D
:103E900000F098FC6B4680B2D880002809D06A46B2
:103EA000074B01A91B889380064B0022188803F05A
:103EB0009DFD3FB000BDC0463461FF1F3561FF1F4F
:103EC0000641FF1F1042FF1F00B50C4BBFB01A7810
:103ED0000B4902A801F0D0FC6B4680B2D8800028C4
:103EE00009D06A46074B01A95B8D9380064B0022DF
:103EF000188803F07BFD3FB000BDC0465E61FF1F28
:103F00005F61FF1FAC40FF1F1042FF1FF7B50E009F
:103F1000377A1C0008AB11003D001A8820231D4091
:103F20001F423CD13378022B3BD173681F785B78FA
:103F30001B023B431E4FBB4208D01E4FBB4214D056
:103F40001D4DAB4221D00A252800FEBD002A2AD1F2
:103F5000142C2AD82200F06807F0DAFB174B1C70EB
:103F6000012CF1D9FFF7B0FFEEE7002A1BD1202C7E
:103F70001BD82200F06807F0CBFB114B04211C700A
:103F8000104B187807F074FBDEE7E3B201240092CF
:103F900001940A00310007F0DDF80500D4E7082598
:103FA000D2E70125D0E70B25CEE70D25CCE7C046AB
:103FB000F3FF0000F4FF0000022900005E61FF1F14
:103FC0003461FF1FE061FF1F332310B5040003704D
:103FD0000A220749013007F09BFB064B0F201B68A4
:103FE0001A0AE37222731A0C1B0E6273A37310BDBC
:103FF000A861FF1FD061FF1F30B5012503790400C0
:10400000BFB02B4213D00B49408806F00FFC28426A
:104010000DD06A46084B02A81B889380FFF7D4FF97
:104020006B46D8800022608801A903F0DFFC3FB016
:1040300030BDC0465661FF1F0641FF1F10B5024844
:1040400004F056FB10BDC046F93F001170B51600D4
:1040500004AA148805AA15784A68507811780002D5
:104060002A4A0843801805284BD807F0E9FA0313B9
:104070001E29343F0720042C0BD80522121BAA420C
:1040800000D92A0022491A803000091907F040FBA4
:10409000002070BD0720112CFBD81222121BAA424F
:1040A00000D92A001B491A80EEE707200E2CF0D811
:1040B0000F22121BAA4200D92A0017491A80E3E7EF
:1040C0000720032CE5D80422121BAA4200D92A009B
:1040D00012491A80D8E70720032CDAD80422121BD1
:1040E000AA4200D92A000E491A80CDE70720032CE6
:1040F000CFD80422121BAA4200D92A0009491A80EB
:10410000C2E700220A201A80C3E7C046DCD5FFFFC1
:104110003BB900117C61FF1F2BB9001126B90011BA
:1041200021B900111CB9001110B50D21024A034834
:1041300006F0F4FA10BDC04610B900111C41FF1F73
:10414000F0B50024274E85B03000B47100F0E2F8DD
:10415000254D264BEA89297C9A422FD10423300031
:1041600003AA00F057F90400300000F011F9012310
:10417000B371002C34D16B4699892B68C9BA4B4373
:1041800029891B4A1B145B1853806B46D9896B68BD
:1041900049BA89B24B4369891B0C5B181548191C35
:1041A0001BB2834200DD011C0B0400D500211388E3
:1041B000918001331380200005B0F0BD022722005A
:1041C00003AB3000009700F0F7F80E230400297CC1
:1041D0000122300000976B4400F0EEF80443C3E77F
:1041E0001C00E8E7F441FF1F9061FF1F83050000FA
:1041F000A861FF1F0F27000073B5234E300000F0A9
:1042000089F8224D07236A463000297C00F002F924
:1042100004003000002C33D16B461B787F2B2FD845
:1042200000F0B6F86B46D878F02302041B031A405E
:104230006B469B8816495BBA9BB21A432B680009F0
:1042400053432A891B0C9B184B806B465A789B78EA
:1042500012031B011A436B68024353436A891B0C08
:104260009B180C481A1C1BB2834200DD021C13046D
:1042700000D500220B888A8001330B80200076BD98
:1042800000F086F80124F9E7F441FF1F9061FF1F59
:10429000A861FF1F0F27000070B5114C237C002B75
:1042A0000FD0382B0ED10F4D280000F033F8CC235F
:1042B000AC222800217C9B0100F0F4F8280000F0DB
:1042C00067F870BD084BE2899A42FAD1054D280083
:1042D00000F020F800222800217C00F0C5F8EDE76E
:1042E0009061FF1FF441FF1F8305000010B5084BCC
:1042F0001A7C002A09D05B69002B06D09847041E5F
:1043000001D0FEF77DFE200010BD0124F9E7C04674
:104310009061FF1F70B5C17905000C00631E9C41C0
:104320001A4BE402E41849000460C9B2007905F0B0
:10433000DFFEE979687949000131C9B205F0D8FE9C
:10434000E8790930C0B206F0A3FF0023E3666133C9
:104350002360AA795B3B002A0ED022689A43023B75
:10436000134323600A23E36107332362002323639B
:10437000A3630133E36370BD22689A4302231343AE
:104380002360462363610633A361EFE700500040DA
:1043900070B5002504000368DD66C0790930C0B23D
:1043A00007F06EF82900207905F03EFE29006079BB
:1043B00005F03AFE70BD0000F8B51E0006AB1D7892
:1043C000002304681700E366616007F081F80123A9
:1043D0008022E3662B0027615200013B08D207F0E0
:1043E000AFF908200A4A1168002D03D12800F8BD52
:1043F0002261F2E7236F034203D02369013D33704A
:10440000013613685B1A032BEED90125EEE7C0468F
:104410006008FF1F70B51C00002305681600EB66DE
:10442000696007F055F801238022EB6623005200F3
:10443000013B08D207F084F908200A4A1168002CD1
:1044400003D1200070BD2A61F2E72B6F034203D035
:104450002B69013C3370013613685B1A032BEED9CC
:104460000124EEE76008FF1F002370B50468150003
:10447000E366616007F02CF80123E366256107F02D
:104480005FF98020064A80001168636B034205D102
:1044900013685B1A032BF8D9012070BD0020FCE7DC
:1044A0006008FF1F70B51D00002304681600E36656
:1044B000616007F00DF80123E36626610F33626B3C
:1044C0001A42FCD02B0A23611023626B1A42FCD0E3
:1044D000EDB2256107F034F98020074A80001168A9
:1044E000636B034205D113685B1A032BF8D90120D3
:1044F00070BD0020FCE7C0466008FF1F10B5084CE7
:10450000E368002B08D18022064B52021B689B18DF
:104510006360054B1B68236007F03AF9A06010BD8B
:10452000D061FF1FC8F00040CCF0004070B5184AC1
:10453000936A916A9942FBD116498A689A421FD3BD
:104540009A1A8B60144B0126186893B2D202D20ECD
:104550004343424300204C681B0A1B1912029B185C
:104560000E4C0A684B60551CA3420CD8002801D0A1
:104570004B600A600A4A136008680A4B186070BDF5
:10458000581E821ADDE7084A30009B182A00EAE725
:1045900000F00040D061FF1F140AFF1F40420F00CF
:1045A000C8F00040CCF00040C0BDF0FF70B51F4C1B
:1045B00023793F2B01D93F2323711D4B22791A7098
:1045C0001878C0B207F00CF918231A491A4A0B8060
:1045D0001A4913800B805380A379194980200B80DE
:1045E0000C21938001334B43164D191C000183426B
:1045F00000D9011C2980D1806379002B11D10133AE
:104600006371237A012B01D8022323726279237A02
:104610000D4853430A21584306F0D2FE0B4D286043
:1046200070BDA02BEDD9A023EAE7C046C461FF1FEF
:10463000480AFF1F0E42FF1FD043FF1F0C42FF1FFF
:104640000A42FF1F0842FF1F71020000B461FF1FF2
:10465000F8B515210020FEF7C1FE114C011E114DC9
:1046600009D10C22104BC1CBC1C4280006F010FFA9
:10467000FFF79CFFF8BD0C2220000C49FEF782FEDC
:104680000C2802D0084B43CB43C40C222800084915
:10469000FEF778FE0C28EBD00C220021E5E7C0469F
:1046A000C461FF1F9061FF1F80B90011FC0C000066
:1046B000F50C0000F0B51D4C8022A54404008820B4
:1046C00069465201400507F0ABF8902212016A4496
:1046D0001300200032C832C316C816C38023144CFE
:1046E000144FA6689B033343A3603B6006F018FF9A
:1046F0008823A0685B05C01806F0B2FE0025882359
:1047000029008022A0685B05C01840196944520046
:1047100007F07EF880230135FF355B019D42EED125
:10472000A6603E60044B9D44F0BDC046FCEFFFFF19
:104730004043FF1F9808FF1F04100000F0B504005D
:1047400087B0002825D0684606F042FE1B4C0228A0
:1047500006D106226946200006F07AFF002816D00E
:104760006946002301250F262F00E25C0133100962
:104770001030874038002F00324097403A00024303
:104780004A610439062BEFD16846FFF793FF07B063
:10479000F0BD182269460A4807F042F86A46A300AD
:1047A000D358013305D01822FF21684606F070FE69
:1047B000EAE70134062CF1D1E9E7C0466509FF1F9D
:1047C00000090011F0B5002504000E0085B0AA42D2
:1047D00000D183E04B1C087801934B7889783779B6
:1047E00009021943F3783F061B040B431F43039749
:1047F00020706570252800D193E033D8112813D894
:1048000006F0A6FF66000D010D010D010D01A700C8
:10481000B500AE000D010D010D010D010D010D01E1
:104820000D010D01E7000701232800D1C0E0DB28BE
:1048300000D016E1042A00D8A9E01025052A05D0E9
:10484000551F2A003800711D06F062FF0522310055
:10485000200006F05DFF2A003900601D06F058FFB9
:1048600005353BE0562856D010D8332800D19AE0C1
:10487000552836D02628DAD1894B29001322180072
:104880001D0006F005FEFEF7BBFB59E0712800D1C4
:1048900074E0722800D17DE0DC28C8D1022A00D85B
:1048A00075E07378BFB26370B378A370032A05D044
:1048B000033A390092B2F01CFEF79EFC1022390038
:1048C000E01CFEF75FFDC51C002807DA60705CE0A5
:1048D0000C222000734906F01BFF0C25280005B0B0
:1048E000F0BD013A704D0C2A13D8002A0AD02800D6
:1048F000019906F00DFFFFF759FE0C2228006B49C5
:10490000FEF77AFC29000C22601C06F001FF0D2541
:10491000E4E70C22EBE7644D654B2A0043CB43C22E
:10492000E9E7013A5E4D0C2A11D8002A08D0019916
:10493000280006F0EDFE0C2228005E49FEF75CFC24
:1049400029001322601C06F0E3FE1425C6E70C22A2
:10495000EDE705225849601C06F0DAFE0625BDE7A2
:1049600012225649601C06F0D3FE1325B6E7082232
:104970005349601C06F0CCFE0925AFE77178F02999
:1049800005D8504B188801F0D3FB0225A6E7FF237A
:104990006370FAE74C4B012A03D072785A70627048
:1049A000F3E75B78F4E72000FFF70EFB050095E7DF
:1049B000042A04D9454D2F6006F0EAFEA860FFF7EF
:1049C000B5FD0422039003A9601C06F0A1FE052595
:1049D00084E73F4D062A15D906222800019906F0E2
:1049E00037FE00280ED006220199280006F090FE1E
:1049F000062238492800FEF7FFFB0123324A51788E
:104A00000B43537029000622601C06F081FE072527
:104A100064E7012ABBD07078FFF790FEB5E7012864
:104A200000D004E7931E2C4F132B04D87378002B6F
:104A300009D100F009F9294B39001D78601C6A1E64
:104A400006F066FE4AE7551E2A000199380006F076
:104A50005FFE2349AAB23800FEF7CEFB00F02CF926
:104A6000E9E7DA2893D1042A91D9082A15D9B3792C
:104A700072791B021343F27912041A43337A1B062C
:104A800013433B603B68052231002000039306F08E
:104A90003FFE0422601D03A96CE7FE236370F1E76B
:104AA0009061FF1F8CB90011C461FF1FFC0C000056
:104AB00080B90011F50C00009C61FF1F7C61FF1F95
:104AC0004443FF1F1042FF1FC061FF1FD061FF1F43
:104AD0006509FF1FADAC0000C163FF1FBF63FF1F6F
:104AE000AEDE000070470000020010B5094B0A322C
:104AF000094C92B2DA815A8298811882207802F0A9
:104B00007DF90422054B012120781A7006F0B0FDD2
:104B100010BDC046CE42FF1F0A64FF1F0964FF1F7D
:104B2000013870B5042809D806F08AFD0309230866
:104B300012001E4B0221187806F09AFD70BD1B4B27
:104B40000821187806F00CFE0022194B1A72F5E7BE
:104B500080220024164B154D52001A810821287816
:104B60001A68DC7206F054FC2100287806F028FE52
:104B7000E4E70E4B0821187806F0F2FD0D48FFF728
:104B8000C1F80D4B0D4A9B7993800D4A138000228A
:104B9000074BDA720132FF321A810A4B5B78002B25
:104BA000CCD0094A136006F02BFEC7E7E061FF1F77
:104BB000B461FF1F1942FF1FC461FF1FD043FF1FD5
:104BC0000A42FF1FC061FF1F34F0004010B50029EA
:104BD00005D1082803D10131013005F053FA10BD89
:104BE00010B501290FD108280DD10021013005F0A1
:104BF00049FA054B1B78002B05D02622034B0448AD
:104C00005A72FFF771FF10BDE263FF1FB461FF1F0F
:104C1000C40900000300F0B50A4D8E18B14202D15C
:104C200052008018F0BD0C782F6824093C5D0F27D6
:104C30001C700C7801313C402F683C5D5C70023385
:104C4000ECE7C0460442FF1F0E22124B10B51A704B
:104C50000D23114C11492370093A043B104863702D
:104C600006F056FD2D2301220E490F48E371FFF790
:104C7000D1FF01220D49FFF7CDFF01220C49FFF7BB
:104C8000C9FF030000200B4902001870FEF7B4FAB8
:104C900010BDC046DE63FF1FBF63FF1F3BB900119D
:104CA000C163FF1F6709FF1FC763FF1F6609FF1F5F
:104CB0006509FF1FAEDE000070B5124C1422200003
:104CC0001149FEF75FFB431E104D132B17D8AB782D
:104CD000002B14D0431C2B7009236B700023001988
:104CE0000370287829000130C0B206F0A1FD2978B0
:104CF00022000139C9B2002005F02EFC70BDFFF77B
:104D0000A3FFEEE7C163FF1FAEDE0000BF63FF1F1E
:104D100010B5114B1A781870002A0ED000280BD14C
:104D20000E4B1A78062A07D85423D340DB0703D545
:104D30000B4B187802F062F810BD0028FCD0074B2E
:104D40001B78012B02D0033B022BF5D8044B012129
:104D5000187806F08DFCEFE7E263FF1F0964FF1F80
:104D60000A64FF1F70B5504E504A514930700820F8
:104D700005F07EFA0121092005F084F9092005F0EB
:104D800065FA0121002005F07DF9002005F05EFAAA
:104D9000FEF736F906F0BCFB032246494648FFF70A
:104DA00039FF2D24030004221C7044490130FFF711
:104DB00031FF30230470424D424C437083702E3BD0
:104DC000062220004049EB87FEF7DCFA062813D0C4
:104DD000200006F0FDFA022809D00321200006F089
:104DE00067FB8D23E3706E3B2371193363710622D9
:104DF00020003549FEF700FA344B1B68FC335C6435
:104E0000FFF75AFF0020FFF783FF314C314A0121A1
:104E1000314B1278207801F0B3FF304A304B1278D2
:104E20000021207801F0ACFF01222E4B1A702E4B8E
:104E30009B78552B31D12D4B3B325A722C4B2D4A3E
:104E4000AB81EA812B826A822021307806F090FCC7
:104E50000120404205F0CCFB0120404205F068FCF7
:104E6000FFF762F9FEF716FF00F09EFC01204042BA
:104E7000FEF7ECFF012006F06BFAF02001F03CF9A0
:104E80000121307806F0F4FB307802F013F91A486B
:104E900006F09EFCFEF712FE70BD6422174B5B7994
:104EA00053431A000A32CBE7E061FF1FCD4B0011DC
:104EB000E14B00114443FF1F7C61FF1F9C61FF1FFA
:104EC000CE42FF1F6509FF1FADAC00002C64FF1F21
:104ED0000A64FF1F3842FF1F1942FF1FDE63FF1FD6
:104EE000BF63FF1FB063FF1FC061FF1FB461FF1FDF
:104EF000C4090000CE090000E261FF1FC461FF1F6A
:104F0000F8B50A0020230D001A40194251D0544B25
:104F10001B78002B3CD0FFF709FB524B524C534EF1
:104F200099686268737A8A1ADB039A4202D36160D5
:104F3000FEF7C4FD327A217A531EDBB299422AD1A0
:104F4000FFF7AAF9637A002B1FD0013BDBB2637233
:104F5000002B1AD1464B9B78552B01D106F050FC03
:104F6000E37A002B0CD00023424A434FE3721388AC
:104F7000380001331380FEF7C5FE390006F078FCD7
:104F8000642370795843FFF7AFFD237A013323720E
:104F900020206840F8BD9142D4D300232372FFF74C
:104FA000A5F9354F3800FEF7ADFE390006F060FC7C
:104FB000C8E70BB2002B0ADA304B187806F0E0F99C
:104FC000002801D006F034FB80200002E1E7022433
:104FD000214206D0244B01201A72FFF799FE2000CF
:104FE000D7E70B071BD5FFF7A1FA1E4B1E491F4C35
:104FF00098684A68637A821ADB039A4202D348604F
:10500000FEF75CFDFFF772F9FFF746F900F0E6FBEB
:105010002368DB0701D5FFF711F80820B9E7102452
:105020000E002640214206D00D4B1B78002BD6D116
:10503000FEF744FED3E70124214209D0104800F0D6
:105040006DF806F00DF93100092005F01BF8C6E7F0
:1050500004240800204021429CD0FEF713FFBEE745
:10506000E263FF1FD061FF1FB461FF1FC461FF1F18
:10507000C061FF1FA861FF1F1942FF1FE061FF1FF2
:10508000FC41FF1FF0B51B4B1B4F1B883A880400E7
:105090001A4E1B4D85B09A420DD832889A420AD3D7
:1050A000184B1A882B889A4205D1174A174B128839
:1050B0001B889A421BD0052001F074F83B8802AA95
:1050C00013803388019053802B88114D93800F4BB0
:1050D00002A91B88D3800F4B2A78188802F090FD14
:1050E0000D4B08212878019A1C7006F081FB05B051
:1050F000F0BDC046AE63FF1F0E42FF1F0C42FF1FF4
:105100000A42FF1FAC63FF1FAA63FF1F0842FF1F75
:105110000A64FF1F1042FF1FA863FF1F13B50C4B4B
:105120001C78002C11D1002801D00A4B18600A4AC3
:105130000A4B11780A4A10780A4A01920A4A0092E8
:10514000002205F001F9200016BD1124FBE7C0463E
:105150000964FF1FA463FF1F0864FF1FF863FF1F9C
:105160000A64FF1FE463FF1FE863FF1F10B5064BCF
:1051700012201B78052B06D1044B13221988044BEF
:10518000187801F0EBF910BD0964FF1F1042FF1FF2
:105190000A64FF1F10B500240122114B52421870FF
:1051A000104B1C70104B1A8001F084FF04220F4B2F
:1051B00021001A700E480C3206F03AF91022210034
:1051C0000C4806F035F907220B4B1C600B4B1C708A
:1051D0000B4B1C700B4B1A700B4B1C7010BDC04658
:1051E0000A64FF1F0964FF1F1042FF1F0864FF1FAE
:1051F000F863FF1FE863FF1FE463FF1FBE63FF1F29
:10520000BD63FF1F1242FF1FBC63FF1FF8B5174CA1
:105210000600257806A814240078052D23D1B41F94
:10522000134FA5B21824BD421DD88D1FADB2BD428B
:1052300019D8FA256D00AA4215D21D000D4F0A3D5E
:10524000ADB2BD420FD80C4C26800C4C21800C49CD
:1052500000240A800B4A1380FFF714FF0A4B042135
:10526000187806F07DFA2000F8BDC0460964FF1FDB
:10527000790C0000750C00000E42FF1F0C42FF1F4E
:105280000A42FF1F0842FF1F0A64FF1FF0B50BB25E
:105290000D0089B0002B00DB70E1A44E307806F0E1
:1052A0006FF8041E50D00378A22B00D122E1D02B3E
:1052B0001AD0912B45D143780E2B42D19C4B82883A
:1052C0009A423ED19B4A83681278052A39D103203D
:1052D00018567F2835D0984B1B68002B31D05B685F
:1052E000002B2ED098472CE08078072829D806F08C
:1052F000A7F90428183F3F74A8D86378002B0CD175
:1053000001218C4B19708D4B1A78002A5BD08C4B85
:10531000307801F035FD002855D00722854B1A70F2
:1053200051E061780029F8D1E378002B11D0854A4B
:10533000854B1278307801F023FD60706378002B84
:10534000EBD1200006F074F980200002684009B01B
:10535000F0BD784B1B78022BF3D00121307806F09A
:105360001FF80028EAD10121307806F081F9E5E73D
:105370006378002BD1D16F4F032807D13B78052BE1
:1053800002D101333B701EE00223FBE76F4B1A880A
:105390006F4B0293002A0BD01B78002B03D0012106
:1053A000307806F025FA3B78062B04D1013BE9E77B
:1053B000029B1A70F7E7042B41D10121029B307840
:1053C000197006F055F95C4B1B68002BB9D01B68AF
:1053D000002BB6D0574A107884E76378554F002BDE
:1053E00027D10622211D5B4806F092F962895A4BAB
:1053F0005A491A80A2895A4B1A80E3890B800521E9
:10540000397058490A80584A1380228A574B1A80AB
:10541000574B1B78012B09D11F2000F0C3FEFA2245
:10542000920042430421307806F0E2F90022484B12
:1054300075E7312B00D070E70022454B1A7003232B
:10544000A0E706220021434805F0F2FF0023454A69
:1054500004211380444A30781380444A138006F0B4
:105460007FF90821307806F07BF9A379083B5A428E
:105470005341304A03331370304B1B78002B06D056
:10548000334B30781A78002A06D001F0B7FC01229D
:10549000314B52421A8096E70121197006F0E8F864
:1054A000F5E70821307806F05BF96378002B00D02F
:1054B00047E72C4B2D4F0293E388029A0421138077
:1054C000294B307803932389039A138063893B80A7
:1054D00005F066FF002800D033E7264B1B68002B41
:1054E00000D12EE7039902983A88098800881B6842
:1054F000984726E74379132B00D022E70389012B35
:105500000AD11D4B1B78022B06D10821307806F0FA
:1055100027F9FFF72BFE14E7052000F043FE0821D2
:105520000200307806F064F90BE7C0460A64FF1FFA
:10553000051400000964FF1FA463FF1F3842FF1F0A
:105540001942FF1FDE63FF1FBF63FF1FE063FF1FE2
:10555000E263FF1FB163FF1F1042FF1FB863FF1F0D
:10556000BA63FF1FAE63FF1FAC63FF1FAA63FF1F79
:10557000B063FF1FA063FF1FA863FF1F8020C0014F
:10558000014200D0E2E6CB0731D5324B1B78002B2D
:105590001DD0314E05AC3378052B1AD1023B237058
:1055A0002E4B21001B7823722D4B1B7863722D4BE1
:1055B000187801F089FB002809D007202A4B3070A9
:1055C0001B68002B03D01B68002B00D098470120DC
:1055D000BCE60E20254B06221B7825492370254B5F
:1055E0001B78637002ABC01806F092F8D8E702236C
:1055F00008001840194209D0174B1B78052B03D11E
:105600001D4B188805F06CFF02209FE60424214200
:1056100003D0FFF737FD200098E608230800184064
:10562000194200D193E6154B1C78012C03D0022CB3
:105630000DD008208AE6124B124A134913481B88E2
:105640001288098800880094FFF7E0FDF1E7FFF772
:105650008DFDEEE7E263FF1F0964FF1F1242FF1F8B
:10566000BC63FF1F0A64FF1FA463FF1FBE63FF1F0D
:105670001342FF1FBD63FF1F1042FF1FA863FF1FE0
:105680000842FF1F0A42FF1F0C42FF1F0E42FF1F6E
:1056900010B502A804880B20002C10D149680878A6
:1056A0004978090201430C48814209D1022119803D
:1056B0000A4B59881170DB7800205BB2537010BD23
:1056C000074C0A20A142FAD102211980034B998884
:1056D00011705B79F0E7C0466E2A0000A861FF1FD9
:1056E0006F2A0000F7B5150008AA16884A680F4F00
:1056F00014785278120222430A24BA4214D10122A9
:10570000DBB2019200962A0005F024FD041E0BD1A5
:10571000074B1B68002B07D068782A7800021043DB
:1057200042425041013098472000FEBD022900004E
:105730001C64FF1F30B5012503790400BFB02B4264
:1057400025D01449408805F071F828420CD0124B3E
:1057500001A95B8D00220B8002234B800F4B5B88DD
:105760008B80608802F042F90D49608805F05EF890
:10577000C0070CD50B4B01A91B8800220B8002230C
:105780004B80064B9B888B80608802F02FF93FB0DE
:1057900030BDC0461464FF1F3C42FF1FA861FF1FBD
:1057A0000C64FF1F9642FF1F10B5074C07492000ED
:1057B00004F0F2FF2000064904F0EEFF0721054A3D
:1057C000054804F0ABFF10BDFFFF00001464FF1F8D
:1057D0000C64FF1FACB900113C42FF1F10B502481A
:1057E00002F086FF10BDC046355700110200F0B52B
:1057F00001270A480A4E51188B1A002B00DCF0BD15
:10580000082415784308684038404000805B013C1C
:1058100058406D08002CF5D10132EDE7FFFF000084
:10582000C6B90011F0B500250F269D4200DBF0BD82
:105830004C5D070944403440A400A058013578402D
:10584000F3E70000F0B589B06A460D000B000F27A2
:10585000110010351C780133260024093E401670D3
:1058600054700232AB42F5D12023024AFFF7DAFF2F
:1058700009B0F0BDCCB90011F0B54E780B7889B005
:1058800036020C00170001901E43012A61D9954B86
:105890009E4200D877E001339E421CD1062A17D1E0
:1058A000CA788B7812021A430B791B0413434A7986
:1058B00012061A438C4B5A6100221A705A808B4A86
:1058C0005A608B4A9A608B4ADA60002009B0F0BDBA
:1058D00088225205EEE7884B9E423CD182498B7864
:1058E000002B00D0F6E00C2A31D10F22A37893438D
:1058F000E2781202134322791204134362791206EA
:1059000013434B60E279A07912020243207A00042B
:105910001043627A12060243CA60E27AA07A120247
:10592000024376484A81834208D804236E491422F0
:1059300001980B7005F0ECFE1420C7E71201D21895
:1059400089235B059A42F0D801238B70BDE7022AB8
:10595000FAD00523EAE76A4A01239642E6D1FFF727
:1059600005FC052F0CD9E378A2781B02134322799A
:1059700012041A4363791B061343624A03931360AC
:1059800005F03EFFA1E7584D2B78002B9DD1AB7859
:10599000002B00D1A0E02B8901339BB20093B342CE
:1059A00000D091E0132AD4D9CF7C8B7C3F02122106
:1059B00020001F43FFF71AFF874200D08EE0002E21
:1059C0003DD1E378A2781B0213432279E9681204DF
:1059D0001A4363791B06134303930A228B4212D1A5
:1059E000FF23A370E370237163716B89002B09D1CE
:1059F000E37B227C1B0212041343A27B13431B098B
:105A000001336B8100226B89002B8ED0002A67D175
:105A1000686837013818000B6B69000303909842DF
:105A200005D9686105F01CFDEB780133EB706868FF
:105A30001022A11C381805F0EBFE2E8145E76F8976
:105A4000009A7B1E9BB293423AD1E278A37812026D
:105A50001A43237905A81B04134362796C68120664
:105A60001A43EB6800920392211D0C22049305F067
:105A70004FFE0120260004A940421036FFF7E2FE47
:105A8000013F012F17D1009A0B232861824200D0D9
:105A90004CE704221C49200005F0BAFE042203A9A9
:105AA000686805F0BDFEE968039AFF23914200D1C2
:105AB0003CE7F73B3AE73100FFF7C4FE1036DFE77B
:105AC0000923B742A4D831E7009BB34200D9FCE6D2
:105AD00007232BE7022329E7032327E7062325E7EC
:105AE0000A2323E7FFFE0000B042FF1F0000011160
:105AF000FFFF00005048593601FF0000FFFF001172
:105B000002FF000034F00040BC42FF1F10B5034C00
:105B10000B000122210000F06BFA10BDCD5C0011DA
:105B20000B8870B506000D000224162B11D92B002E
:105B30000322094900F05CFA041E0AD1074B2A88A7
:105B40001B88191C934200D9111C300089B200F047
:105B5000EFFA200070BDC046F95C00114664FF1FDB
:105B600010B54A780400013A0B000220012A07D838
:105B70000A78002A04D005222000024900F038FAF1
:105B800010BDC046275D00110A7810B50B00040057
:105B90000220002A04D007222000024900F028FA3F
:105BA00010BDC046D35D00110A7810B50B0004008B
:105BB0000220002A04D009222000024900F018FA2D
:105BC00010BDC046395E001110B5034C0B000B220E
:105BD000210000F00DFA10BD695E001110B5034CF4
:105BE0000B000D22210000F003FA10BDDB5E001156
:105BF00010B5034C0B000F22210000F0F9F910BD85
:105C0000355F00110A7810B50B0004000220002A4D
:105C100004D011222000024900F0EAF910BDC0466C
:105C2000455F0011002310B51322190000F0E0F9C0
:105C300010BD000010B5034C0B001722210000F02E
:105C4000D7F910BD975F0011002310B51922190074
:105C500000F0CEF910BD000010B5034C0B001B2264
:105C6000210000F0C5F910BDD15F0011F7B584899E
:105C70000D0006000121002C22D000238268D3569B
:105C80001778002B1EDA0C2C1AD90C3CA4B213196D
:105C900040880093230002F086FE431E98410130A5
:105CA0007B06DB0F6B703F23013C1F40A4B22870C2
:105CB000AF70AC80002C07D0B3680133AB6000211B
:105CC0000800FEBD0020EBE7AC60F8E70B7803703E
:105CD0004B8843704B881B0A83700B79C370042078
:105CE00070470420022B06D10020537811781B0244
:105CF000009A0B43138070470B8803700B881B0AB4
:105D00004370022070470420009983420AD15378DF
:105D100010781B0203430B80D37890781B02034357
:105D200000204B807047F8B50D004B78012400210E
:105D3000461C03702B788B4201D82000F8BD6B788D
:105D4000B01C4F1C012B10D1890069184B8802220E
:105D500033704B88B9001B0A7370691805F0B0FCEA
:105D600004360434A4B2F9B2E4E7122359436B18A1
:105D70005A88043132705B8810221B0A73706918CC
:105D800005F09EFC12361234ECE770B5049D140049
:105D90001E00052B01D8042070BD637812781B0209
:105DA00013432B80E378A2781B02134302226B80FB
:105DB0002A71211D681D063E05F082FCB2B22A81BF
:105DC000E92AE8D82800A11D0A3005F079FC002056
:105DD000E2E7002310B50A789A4201D8900010BD7E
:105DE0009A008A185488013304705488DBB2240A5C
:105DF0004470948884709288120AC2700430EAE772
:105E000010B51100029C062B04D004201022142B84
:105E100001D010BD022222714B7808781B02034387
:105E20002380CB7888781B02034363800431601D94
:105E300005F046FC0020ECE710B50C788B780431B7
:105E40005C43E4B203702200013005F039FC601CB1
:105E500010BD0420022B06D10020537811781B02BC
:105E6000009A0B431380704710B50C000A8802316A
:105E700005F026FC208810BD70B504000D000498C4
:105E80001100012B01D8042070BD1678527812023F
:105E9000324302800200F13255701470E125002C6B
:105EA00000D10C35023B9AB24280AA42EBD80231B3
:105EB000043005F005FC0020E6E704200099834249
:105EC0000AD1537810781B0203430B80D378907863
:105ED0001B02034300204B80704710B50C000A885A
:105EE000023105F0EDFB208810BD000070B50121E6
:105EF0001E000420049C0E400B4218D1CB40DDB2A2
:105F00008D4214D90A49DBB2098899420FD3230084
:105F1000EE331D703300580011184978165C0902E1
:105F2000314301332152D9B28D42F4D8002070BDE3
:105F3000C842FF1F10B50C000A88023105F0C0FBF3
:105F4000208810BD10B50C788B7804315C43E4B226
:105F500003702200013005F0B3FB601C10BD10B5CA
:105F600011000298032B01D8042010BD1478527838
:105F7000043B120222430280CA788C781202224328
:105F800042809AB28280EB2AEED80431063005F0C6
:105F900097FB0020E9E710B50C000B8803700B8815
:105FA0001B0A43704B8883704B881B0AC3708A8816
:105FB0000430063105F084FBA088043080B210BDA7
:105FC0000420012B03D100201378009A137070472E
:105FD00010B50C000B8803700B881B0A43704A88AD
:105FE0000230043105F06CFB6088023080B210BDD5
:105FF000F0B589B003931E4B029242000700D05ABD
:10600000019102F020F81325061E2DD0029B0124D9
:106010000370019B002B04D00019039998470019C5
:1060200084B26B461B7A5BB2002B0FDA102138006A
:1060300002F01CFB1925002813D130003219E1B2FF
:1060400002F066FC051E0CD10C34A4B2042304AA91
:10605000380005A993800696948101F0AFFD051ED6
:1060600002D0300005F0A4FB280009B0F0BDC04606
:106070004464FF1F70B505000C0000280CD0002000
:10608000814209D010222000044905F019FB0120AB
:106090002B7823736B78637370BDC0460CBA001104
:1060A000F0B506000D0017001C0085B002291BD0BA
:1060B0000020102907D1022B07D0102B03D115E0A7
:1060C0000020102C08D005B0F0BD69463800FFF75D
:1060D000D1FF2A0069460BE069463000FFF7CAFF8E
:1060E00022006946380004E0022BE9D12A00390079
:1060F000300005F055FBE6E7031CF02800D9F0233B
:10610000032008499AB2013A0B80D317034006498D
:106110009B189B100B80D30F04499B185B100B80BE
:106120007047C046CC42FF1FCA42FF1FC842FF1F34
:10613000034B1B888B4202D3024B4000C152704775
:10614000CC42FF1F4464FF1F014B4000185A7047A8
:106150004464FF1F1722014B1A8070474464FF1FDD
:1061600070B505000E2005F013FA041E13D0D023DD
:10617000037000230622837007494570033005F041
:106180009FFA064B2100DA8A62811B7E2373044B3F
:10619000187805F0BDF870BD6064FF1F5064FF1FE4
:1061A0001C43FF1F262803D8024B4000C05A7047EB
:1061B0000148FCE7CE42FF1FFFFF000070B506005C
:1061C0000C00094D1C220021280005F031F9074B75
:1061D0001E70074B1C7005F023FA0123002801D024
:1061E000002312202B7070BD5064FF1F1C43FF1F43
:1061F0007164FF1F70B505000D4C0800E260A160DE
:1062000010220021656005F03BF8012803D1102120
:10621000A06802F058FD10220021280005F030F897
:10622000012803D11021606802F04DFD70BDC04609
:106230005064FF1F70B5041E05D1002903D006224B
:106240000D4805F03DFA0D4B1D78012D11D1002CA4
:1062500005D102221A7005F053FA280070BD002201
:106260001A70074B1B78FF2BF7D02000FFF778FF41
:10627000F3E70025F1E7C0466064FF1F5064FF1F8D
:106280001C43FF1F030010B5002801D1002010BDE2
:1062900000780B4A002803D15988D1821B791376E4
:1062A0001378022BF2D10023984200D103331370EC
:1062B000044B1B78FF2B01D0FFF752FF0120E6E7CC
:1062C0005064FF1F1C43FF1F002911D000280CD071
:1062D0004B79012803D140225242134303E03F226D
:1062E0001340032802D001204B7170474022F4E78D
:1062F0000800FAE770B5094D0100287800280BD096
:10630000074C0622200005F0DBF921002878FFF772
:10631000DBFF200005F004F870BDC0467064FF1F6D
:106320004A64FF1F00290AD0012808D13F224B7977
:106330009343C02B03D0403B5A425341981C7047B3
:1063400070B5174D06002B78FF2B15D00A2005F0ED
:106350001FF9041E10D0D0230370C83B8370114B6B
:1063600011491B784670C3700622043005F0A8F965
:106370002100287804F0CCFF0C4B1B78012B0DD1A9
:106380000B4B1B68002B03D09B68002B00D0984759
:10639000084B04211878084A05F03AF870BDC04649
:1063A0001C43FF1F7064FF1F4A64FF1F6C64FF1FC4
:1063B0009864FF1F9C64FF1F60EA0000014B98680F
:1063C0007047C0465064FF1F014BDB681868704778
:1063D0005064FF1F074B10B5DA6813680133136070
:1063E000054B1878FF2803D08021C90105F040F93A
:1063F00010BDC0465064FF1F1C43FF1FF7B50E00C1
:1064000002F0C8F8051E1CD00E4B06621F78002F44
:1064100000D10778AB791020019305F0B9F8041E7C
:106420000FD0D0230380C73B8370019BE91DC3704D
:106430000622043005F044F921003800E66004F03B
:1064400067FFF7BD1A43FF1F014B18787047C0461E
:106450007064FF1F054B002805D1054B1A78054BCA
:10646000002A00D1014B18007047C0466064FF1F2E
:106470007064FF1F4A64FF1F014B58687047C04695
:106480005064FF1F024B1868431E9841C0B270470A
:106490007464FF1F421E03000120152A03D9FF3B2D
:1064A0005A425341D8B27047F0B51C0000230E0089
:1064B00085B0039002920B70029A934201D30020A0
:1064C00019E0E55C5A1CD2B2002DF8D0029851199F
:1064D0008142F4DC0233DFB2A35C18000193FFF7C2
:1064E000D9FF002807D0013D019A0399EBB2337020
:1064F0008A4202D1E01905B0F0BDDB19DBB2DBE75F
:1065000010B50C0002F09EF803001220002B03D0FF
:106510002100588804F024FF10BD000070B50E4D16
:1065200084006359002B15D0186A002801D004F0AC
:10653000FFFE2B59586A002801D004F0F9FE2B59B0
:10654000986A002801D004F0F3FE285904F0F0FE08
:1065500000232B5170BDC0468064FF1F1C4B70B5DB
:1065600004000E00150099420AD11A4B1B68002B3B
:1065700001D1122070BD1B68002BFAD09847F9E7B3
:10658000154B994215D1134B1B68002B0AD01B6881
:10659000002B07D09847002804D1104B1C70104BDB
:1065A0001D70E7E729002000FFF7AAFF0028E1D1CE
:1065B000F3E7080001F0EEFF0028DAD003780320AB
:1065C000A342D7D12900300004F0CAFED2E7C0466A
:1065D000FEFF00007C64FF1FFFFF00007964FF1FC7
:1065E0007864FF1FF7B50400808801F0D3FF002511
:1065F000A84203D00578A08802F008F81C4E337832
:10660000002B1FD0AB421DD11A4B28001978FFF781
:1066100077FF002818D000233370A3790820A778CB
:10662000A688019304F0B4FF011E0DD0D02303709F
:10663000CA3B8370019B477086808371280004F0F9
:1066400067FE01E0002DE8D1A0880B4B8200D358F3
:10665000002B01D0FFF762FF1721A088FFF768FD2C
:10666000A08801F027FDA08801F0FEFDF7BDC0461F
:106670007964FF1F7864FF1F8064FF1FF0B587B047
:106680001D000CAB1B88070001930DAB1B88142069
:1066900002930EAB1B88160003930FAB1B8800916F
:1066A000049310AB1B88059304F072FF041E1AD0EC
:1066B000D0230370CB3B47708370C670062229003D
:1066C0000430002D11D004F0FBFF019B21006381F9
:1066D000029B0098A381039BE381049B2382059B7B
:1066E000A37404F015FE07B0F0BD04F0A1FEECE7C2
:1066F000F7B5009308AB1B8807000C200D001600AF
:10670000019304F045FF041E13D0280001F042FF5E
:1067100000280FD00078D0232370C93BA370009BC2
:1067200021002381019B6770A580E680638104F0CE
:10673000EFFDF7BD014B1878EDE7C0461C43FF1F86
:1067400013B5040064890389C2888188C0780094E5
:10675000FFF7CEFF13BD000010B5044C20680028E1
:1067600003D004F0E5FD0023236010BD8464FF1F07
:10677000A122F0B5818892004A43384B384F1B68FC
:1067800004009B189D2292009B18827989B01A60A0
:106790003B68002B5FD01D78324B1B68002B04D068
:1067A0005B68002B01D00020984726000836310096
:1067B000E079FFF7B7FD237DE0710200E0780493F4
:1067C000638A29000393238A0293E3890193A388B0
:1067D00000933300FFF752FFE378002B0BD1E289DF
:1067E000A379A18802920196E27928000092012201
:1067F00001F0DAFEE0703B68002B20D0FFF7ACFF21
:10680000194D287800281AD0184B1978FFF778FE10
:10681000002814D02B78E67808200793A78804F086
:10682000B7FE011E09D0D0230370CA3B46708370A7
:1068300087808671079804F06BFD00232B70172169
:10684000A088FFF775FCA08801F034FCA08801F057
:106850000BFD09B0F0BD064B9DE7C0463409FF1F94
:106860008464FF1F9864FF1F7964FF1F7864FF1F13
:106870001C43FF1FF8B5070008000E0001F08AFE58
:10688000041E18D02620FFF78DFC051E00D12578A8
:10689000062004F07DFE041E0DD00021062204F027
:1068A000C7FDD0232370C23B21006770A370A68070
:1068B000E8B204F02DFDF8BDF0B585B001930AAB48
:1068C0001B78070002930BAB1B7808000D000092A9
:1068D000039301F05FFE061E22D0102004F058FE44
:1068E000041E1DD01022002104F0A2FD2620FFF777
:1068F00059FC002800D13078D0232370C13BA3700D
:10690000009B21002372019B67706372029BA5802C
:10691000A372039BC0B2E3720C9BE36004F0F8FC2B
:1069200005B0F0BDF7B50D00019001F033FE071E74
:1069300020D00E2004F02CFE041E1BD02620FFF7D2
:1069400031FC061E00D13E78D0232380C53B0622B1
:10695000A370F91DE01C04F0B3FE019B2A006381C3
:106960000123DD401A401D40210022736573F0B2FF
:1069700004F0CEFCF7BD0000F0B585B00290100029
:106980000D0017000A9E039301F004FE041E31D08F
:10699000029B002B2ED1039B02795B0724D5122387
:1069A00013430422002E08D10B99002905D10C991C
:1069B000002902D10D9900291AD01A430D9B22718A
:1069C000002B00D0C9E0002E00D1CFE0002D00D078
:1069D000CCE0606A002801D004F0AAFC1C21300041
:1069E00004F016FE606205E002239A430E33D7E7F7
:1069F00093432371654BBA00D458002C00D1AAE010
:106A0000002E10D0236A002B03D11C2004F0B8FD07
:106A100020625E4BBA00D358186A002803D01C22AB
:106A2000310004F04DFE0C9B002B12D0574CBB00E4
:106A30001D596B6A002B03D1162004F0A1FD68627A
:106A4000BB00E358586A002803D016220C9904F0C2
:106A500037FE0D9B002B11D04C4DBC006659B36A1C
:106A6000002B03D1142004F08BFDB0622B59986ADF
:106A7000002803D014220D9904F022FE380001F002
:106A800089FD051E67D0414BBA00D358002B62D058
:106A90001A6A3420002A00D11C389A6A002A01D0D0
:106AA000143080B20B9A002A01D01C3080B25B6A8D
:106AB000002B01D0163080B204F06AFD041E4AD0CB
:106AC0001822002104F0B4FC2620FFF76BFB019094
:106AD000002801D12B780193D0232370029B200042
:106AE00063700A23294EA370039BBD00A371AB59A9
:106AF000A780196A1830002905D01C22A06004F074
:106B0000DFFD200034307359996A002907D0030053
:106B100014221433E060029304F0D2FD02980B9B20
:106B2000002B08D003001C221C330B992061029318
:106B300004F0C6FD02987359596A002903D0162241
:106B4000606104F0BDFD6B462100187904F0E0FBA4
:106B50003800FFF7E3FC05B0F0BD10220D9B0D9946
:106B60001B69A018236204F0ABFD2CE70B9B002BE4
:106B700000D13FE7012D00D03CE7606A002801D03A
:106B800004F0D6FB1C210B982AE7C0468064FF1F47
:106B900010B5044C2068002803D004F0C9FB002382
:106BA000236010BD7464FF1F0B4B07B51A68002AE1
:106BB00001D100200EBD6946531C01201278073117
:106BC000FFF772FC0028F4D002780123100018406F
:106BD0001A42EED0EEE7C0469064FF1FF0B51F4F9B
:106BE00001203B6887B0002B25D09B78059300F0EF
:106BF000B3FB002821D00A20FFF7D4FA04000B20B1
:106C0000FFF7D0FA164B05001E78731E9E413B68B5
:106C1000F6B2191DD878FFF757FB3B682900DA7ADE
:106C2000043303929A79019302920090330020007A
:106C3000059A04F035FD07B0F0BDFFF7B5FF002859
:106C400005D00620FFF7AEFA04000720D8E7082099
:106C5000FFF7A8FA04000920D2E7C0467464FF1FBA
:106C60007064FF1F70B50A4E040033780D00FF2BCF
:106C70000DD0042004F08CFC011E08D0D02303703A
:106C8000CE3B45708370C470307804F041FB70BD1A
:106C90002C43FF1F70B5040006200D0004F078FCA3
:106CA000011E0AD0D0230370CD3B8370054B447086
:106CB0001B688580187804F02BFB002C01D0FFF7AF
:106CC00067FF70BD7464FF1FF8B5264F06003B6870
:106CD0000D001124002B05D10522234B1B781342F4
:106CE00002D112242000F8BD204A10241268002A84
:106CF000F8D01278002AF5D0DB0719D52B789A1E28
:106D0000012A1AD80C2004F03BFC13243860002818
:106D1000E8D000230A22437029000670023004F0F4
:106D2000CFFCFFF75BFF041E0AD0FFF731FFD9E766
:106D300000F012FB0028E1D1E4E7002BE2D0D0E71D
:106D40000B4B1B78032BCDD11D20FFF72BFA094BE2
:106D500018800028C6D0084B04211878074A04F090
:106D600057FBBFE77464FF1F7164FF1F9064FF1F30
:106D70007064FF1F6E64FF1F9C64FF1F60EA0000C9
:106D8000F7B50193194B14001A78052306000F007C
:106D900012201A4221D0012920D1154B1D68002D47
:106DA0001BD002201F2C18D8002C02D0019B002BD6
:106DB00013D0104B1F221E706E1C0021300004F0F7
:106DC00037FB01992200300004F07AFC31002000EA
:106DD0002C70002F06D004F06BFCFEBD064B122079
:106DE0001D68DCE704F024FDF7E7C0467164FF1F6F
:106DF0009064FF1F2C43FF1F8C64FF1FF8B50F4EDC
:106E000012243368002B17D01B780F3C834213D118
:106E100000250B4F0221387804F0A2FC094B042115
:106E200038781D8004F09CFC074B28001D803368D7
:106E30005C7004F05DFA04002000F8BD7464FF1F6C
:106E40009C64FF1F8864FF1F6E64FF1F70B50128DC
:106E500023D11B4C2388002B03D01A4A1578002D10
:106E600007D0194B1B68002B02D01878FFF7C6FF1C
:106E700070BD3B2B02D93C3B2380F9E7134E022126
:106E8000307804F06DFCFA222388920002215A43E4
:106E9000307804F0ADFC2580EAE70B4B1B68002B33
:106EA000E6D00B4B1B785B07E2D5084B0221187824
:106EB00004F056FC0022024B1A80FFF769FED7E768
:106EC0008864FF1F6C64FF1F7464FF1F9C64FF1FB6
:106ED0007164FF1FF8B51E4D2868002803D004F028
:106EE00027FA00232B601B4E3068002803D004F0E3
:106EF0001FFA00233360184F05243B781800204008
:106F0000234221D0154800F02BFA3B78234213D0BE
:106F1000202004F035FB2860002813D02022002117
:106F200004F086FA202004F02BFB041E306005D00C
:106F30002022002104F07CFA002004E0286804F0FC
:106F4000F7F92C601320F8BD00F00AFAF4E7C04608
:106F50009064FF1F8C64FF1F7164FF1F2043FF1F9D
:106F600010B50A4C23681A1E0ED0002808D1013033
:106F7000587004F0BDF9002805D02368002B02D01A
:106F80000021FFF787FE0122100010BD7464FF1F6F
:106F9000F7B5274E050033680191181E21D05C78A3
:106FA000244F012C30D1FFF7FFFD002825D0200011
:106FB000FFF7F8F80400412814D91F4B0221187874
:106FC0001E4A04F025FA1E4B3C3C1C80022233680A
:106FD0005A703B78002B14D128000199FFF75AFE14
:106FE0000120FEBDFA2292004243002AEED0124B4D
:106FF0000221187804F0FCFBE8E7FFF7D3F8020061
:10700000F3E700233B70EBE73B78002BE8D103204C
:1070100004F0BEFA011E08D0D0230370CC3B4570AB
:1070200083703368187804F073F9FFF7B1FDD7E780
:107030007464FF1F6C64FF1F9C64FF1F60EA000004
:107040008864FF1F10B51749838802008B4220D047
:1070500011D815498B4217D0144900205B1899B2FA
:10706000012907D8926811785A425341D8B2FFF7E4
:10707000F9FD012010BD0E4A00209B1807229BB28B
:107080009A424041C0B2F5E783681878FFF768FF7D
:10709000F0E7836899785A78090218781143FFF766
:1070A00077FFE7E70A20000006200000F8DFFFFF77
:1070B000AFDFFFFF014B18707047C0462D43FF1F25
:1070C00010B5064C207001F041FA207804F088F9E0
:1070D0000521207800F062FD10BDC0469C64FF1FB2
:1070E0000BB273B50D00002B00DBC4E0884B1878A1
:1070F00004F046F9041E0ED00378912B0FD0A22B7A
:1071000000D1A1E0834B1878FF2852D0210004F071
:10711000FFF800284DD180200002684076BD4378FA
:107120000F2B76D013D8052B70D00E2BEAD1808888
:10713000794B98422BD8794B98421BD8784B984280
:10714000E0D1A3681878591CFFF774F838E03E2B9B
:10715000D8D18378032B74D06CD8012B6ED0022B3E
:10716000D0D1704B1B68002B23D05B68002B20D044
:1071700098471EE06C4BC0180C28C3D804F060F888
:107180001DC2C2150BC20B0B0B3223C23C00674B56
:10719000C0180728B6D8664B1B68002B09D01B689F
:1071A000002B06D0200098470AE0A3681878FFF764
:1071B000C7F8200004F03CFAADE7A068FFF762F8DA
:1071C00000289FD0F5E7A3681B78002BF1D0554B22
:1071D0001B68002BEDD01B68002BEAD0210055481E
:1071E0009847EDE74F4B1B68002BE2D01B68002B44
:1071F000DFD021005048F3E7504B1B68002BD8D05C
:107200005B68002BD5D021004348E9E7FFF7EAF996
:10721000CFE780884A4B984203D04A4B984200D02F
:1072200070E7464B1B68002BC3D05B68002BC0D0B7
:107230002100D5E7153B012BBBD963E7FFF798FA8F
:10724000B7E7FFF77DFAB4E73F4B1B78042B07D174
:1072500000236A4613800179408800F0C5FCA8E746
:10726000364B1B68002BA4D05B68002BA1D001001B
:10727000364898479DE7012421420AD0294B1B68D4
:10728000002B04D05B68002B01D000209847012020
:1072900043E78B070AD5264B1B68002B04D05B689D
:1072A000002B01D020009847022036E70421280057
:1072B00008400D4200D131E7254E3388002B21D004
:1072C000013B9BB23380002B1AD1FFF7DBF800287B
:1072D0000AD0204B1C70164B1B68002B04D05B6837
:1072E000002B01D020009847FFF7C6F8694601F04F
:1072F00001FD6846FEF7FEFF1D20FEF753FF3080BC
:1073000004200AE7024B187804F02AFAF8E7C0468E
:107310009C64FF1F2D43FF1F0E2000000120000072
:10732000091000009464FF1FFEDFFFFFAFDFFFFFC7
:107330009864FF1F0C2000000B2000007C64FF1FDE
:107340000D200000132000007164FF1FFFFF0000EC
:107350006E64FF1F6C64FF1F10B501F09BF910BD38
:10736000014B18607047C0469864FF1F0B880020CF
:10737000162B01D817230420014A13807047C046FA
:107380004664FF1F00207047074A030011888142AE
:1073900007D091880020994202D101308000101856
:1073A00070470020FAE7C046A464FF1FF0B58F784D
:1073B00006000D00C5B01E2F15D1FFF7E5FF051E15
:1073C00003D10024200045B0F0BD00223B00310075
:1073D000C078009200F0B2FB0400A81C00F0D2FBC1
:1073E000FF23EB70EEE7264B062403931B78FF2B5D
:1073F000E8D0182FE6D87B08224A013BDB00029236
:107400009A589446002ADDD0029AD3185B68002B64
:10741000D8D00878002802D14B78012B02D106245D
:10742000122FCFD107AFAB88697800976446AA685E
:10743000A047041EC6D1AB78029A5B08013BDB0073
:10744000D318390030005B689847041E0BD1AB7825
:10745000042BB6D0039A310010782200009700F078
:107460006DFB0400AEE76A78002AABD1AA7805A9C3
:107470003B88087130000A704B80FEF747FBA0E79D
:107480003043FF1F1CBA00111D4B37B50500984251
:107490000BD000290AD1FFF777FF002805D1194842
:1074A000FFF772FF002800D0058037BD01291AD1EF
:1074B000FFF76AFF041EF8D001235B420380A37824
:1074C000FF2BF2D0FE2B07D00023E078142200938C
:1074D00029001E3300F032FBA01C00F053FB0123F7
:1074E0005B426380E1E70229DFD1013901F0BEF898
:1074F0000028DAD12800FFF747FF041EDFD1D4E7C8
:10750000FEFF0000FFFF0000022210B5074B5242B1
:107510001A80074801325A809A80DA8000F07EFA99
:10752000044801F025F8002010BDC046A464FF1FE8
:10753000AD730011897400110388F7B50400002BA6
:1075400002D102252800FEBD426802211378254899
:107550005268FEF7A5FD00282ED0234F01253A885A
:10756000002AEFD0802321885B0201259B1A9942D3
:10757000E8DC0C2004F004F8061E31D03B88228899
:107580009C4600231800019561469DB2491989B2B5
:10759000AA421BD8002801D062443A800023300060
:1075A000082208C0210004F08BF8104A1368002B51
:1075B00013D100251660C5E76268022113780C48D4
:1075C0005268FEF76DFD0028C7D1BAE760681D015B
:1075D0004019418101330198D6E71A001B68E6E79C
:1075E0001325AFE78ABA00112E43FF1FA064FF1FC7
:1075F00088BA0011014B18707047C0463043FF1F16
:1076000014230A0010B51A40194204D00122102197
:1076100001F048F810BD4B06F9D401208843400022
:10762000F8E710B514008B0604D50122102101F0F3
:1076300039F810BD08230A001A40194202D14BB292
:10764000002B0FDA102101F02DF8002808D02300BC
:10765000F2331B78002BECD0F1342378012BE8D1E6
:107660000020E6E703208907FAD4E2E7F0B51F001F
:10767000184B85B01C68019002910392002C27D111
:10768000200005B0F0BDA5683301ED186B89019AA3
:10769000934211D3029A93420ED8002F04D10A9B31
:1076A000002B10D12C00EBE73B002978039A686887
:1076B000FEF7F6FC0028F2D10136B6B2A388B34239
:1076C000E1D82468DAE7A3680A9A5B891380E9E7BE
:1076D0000026F3E7A064FF1F37B50C000A8849882D
:1076E0000123914217D3002A15D0651D23792A0062
:1076F00002210A48FEF7D4FC102300280BD023797E
:107700006188208800242A000094FFF7AFFF0A2335
:10771000A04200D0230018003EBDC0468ABA001126
:1077200013B50A0008884988012388420BD800282D
:1077300009D00024137905320094FFF797FF0A233C
:10774000A04200D02300180016BD13B50A00088817
:107750004988012388420BD8002809D000241379D6
:1077600005320094FFF782FF0A23A04200D02300D5
:10777000180016BDF0B58BB003904A8808880E003B
:107780000123824255D3002853D00023012704ACA3
:1077900023700022718813000092FFF767FF051E17
:1077A0003ED02078002835D12B78022B18D1677075
:1077B0006A8983000130E31880005A8069680222D8
:1077C000201803F07DFF23780133DBB22370042BF4
:1077D00019D93B006889013080B2002BD9D01FE055
:1077E00002236370122358436A89231804305A8095
:1077F00069681022201803F063FF23780133DBB29D
:107800002370002BE5D10C4A6B899B185A425341D7
:10781000DBB2DFE76378012BE4D12B78022BC7D0F2
:1078200022780A23002A04D021000398FEF798F951
:10783000002318000BB0F0BD0100FFFF0F4BF0B5A7
:1078400004001868002816D083685D89A54207D80F
:107850008288AE18B44203DA12019A18934201D119
:107860000068EFE71E005F891036A74204D10029A7
:1078700000D00D801800F0BD3300EFE7A064FF1FBB
:1078800070B505000C0008880021FFF7D7FF030042
:107890000120002B04D022002800197AFFF7C1FE36
:1078A00070BDF7B50C00002501902300EE331B7866
:1078B000AB4201D800200AE06B00E65A00213000FC
:1078C000E718FFF7BBFF002802D126800130FEBD7C
:1078D000017A0198FFF794FE002802D03B882380AC
:1078E000F5E70135EDB2E0E710B5040008880021A6
:1078F000FFF7A4FF03000120002B03D02000197A1A
:10790000FFF77EFE10BD0000054B1B68002B01D168
:10791000180004E09A6852898242F6D1988870472C
:10792000A064FF1FF0B50E27002687B0039302ABBB
:10793000FF183E8005001F4B40891400984207D075
:107940002B78013000976A6880B2FFF78FFE06003F
:1079500002212B7818486A68FEF7A2FB00280FD096
:107960006C892000FFF7D0FF002802D0013C0419E9
:10797000A4B2039B002B00D01C80300007B0F0BDE8
:1079800002212B780D486A68FEF78AFB0028E7D1B0
:1079900002212B780A486A68FEF782FB002807D08C
:1079A000002EDED03B88A342DBD17489013CDFE7A7
:1079B0006C89DEE7FFFF00008ABA001188BA001167
:1079C00086BA001110B50C00FFF7DEFC03000220A0
:1079D000002B0AD0002C00D023609B781720FE2BB0
:1079E00003D00138FF2B00D1002010BD73B50D006E
:1079F00001A904001600FFF7E5FF172805D0002EA7
:107A000004D129002000FEF727F976BD01221021BC
:107A1000200000F047FE0028F3D0F6E7014B186085
:107A20007047C046B064FF1F37B56B469D1D01000F
:107A300004000222280003F06BFE2B88B02B0ED12D
:107A40002379122B09D12300FA331B78012B06D19D
:107A50000121608800F0E0F801E01B2BF8D037BD71
:107A600010B5054B0421187000F098F8FFF74CFD95
:107A7000FEF770FB10BDC046B464FF1F0020F0B5D8
:107A80000BB20F0087B0834234DA274B187803F02B
:107A900077FC051E2BD00378A02B25D103AE310037
:107AA000FEF7E4F8041E0BD1B378DB0724D51F4B97
:107AB00006341B68002B03D0310068889847040007
:107AC000A868002801D003F073FE002C08D1184AE2
:107AD000039B1340174A934206D0B3781B2B03D065
:107AE0000121688800F098F8280003F0A1FD8020AB
:107AF0000002784007B0F0BD0F4B1B68002B10D080
:107B0000310068889847041EDAD07378002BD7D1EB
:107B1000B27801A90A704B800C716888FDF7F6FFF6
:107B2000CEE70624F1E7C046B464FF1FAC64FF1F34
:107B300000FFFF0000011200B064FF1FF7B50190C5
:107B4000FC200D0017001E0003F022FD040013208E
:107B5000002C12D0B02320002370089BF422677001
:107B6000658026710830002B08D0190003F0A8FDAD
:107B70002100019803F0CCFB0020FEBD089903F022
:107B800057FCF5E710B5041E06D00078FD2803D891
:107B900003F036FCFF23237010BD00000A1F93B2D0
:107BA00010B504000220032B05D882400020024BB0
:107BB000D1529B189C7010BDD464FF1F0B8870B508
:107BC000043B04000D000220032B0BD801212000F0
:107BD00000F04CFD03001420002B03D029002000EE
:107BE00000F0DEFB70BD000007B51300034A0092F1
:107BF0000A00012100F02CFC0EBDC046257E0011BC
:107C000007B5019203220092024B0A00122100F0F4
:107C100049FC0EBDA37E001107B56B4601AA118079
:107C20000449D88008780633012802D1190003F0EE
:107C30009FFC07BDB564FF1F0C4B10B518700023E7
:107C4000FF210B4A1380138193819380094A53804B
:107C50001370517293819372D174D38213755177DB
:107C600003F036FB00F0FCF910BDC046E464FF1FD2
:107C7000D464FF1FB664FF1FF0B58DB06B460020C3
:107C800003910C229B5E834200DBB0E05D4B1878D1
:107C900003F076FB051E00D1A4E00378902B00D002
:107CA0009DE006AF01004688380000F013FA7968BD
:107CB0000400002900D19CE03B88052B6ED13B8954
:107CC000032B1CD905AC200000F0A2F86288172A0B
:107CD00061D83989131D994231D1796823780431EB
:107CE0000291D90738D5607800F08EF9071E06D0CA
:107CF000002303712378012B08D0132B23D0A8680D
:107D0000002800D178E003F053FD75E06288029905
:107D100009A800F0A6F80290380000F08BF909AA33
:107D20002378387A0192002231000092029A00F002
:107D300012F9380000F064F9029B002BDFD030000C
:107D400000F080F9DBE70378032BD8D16288029931
:107D500009A800F0D6F8DEE7122B13D1029909A882
:107D600000F0B5F8021EEAD127498B88002BC6D057
:107D7000887909A92378019161780091310000F098
:107D8000EAF8BCE7002302AA93833000617809AACD
:107D9000FFF72AFFB3E71D4B0993F6E7042B02D048
:107DA0009A1F012AABD8184A043B9B00995A002914
:107DB000A5D0D218907831003A0000F0AEF8002833
:107DC0009DD13B88042B03D001213000FFF724FF15
:107DD000012C04D1A868002801D003F0E9FC280098
:107DE00003F026FC8020039B0002434018000DB0E6
:107DF000F0BD012800D182E701213000FFF70CFF20
:107E0000EDE7C046E464FF1FD464FF1F01001700C4
:107E10000B7803704B784370CB788A781B0213433E
:107E2000438070470A88030002700A88120A427071
:107E30000A88012A06D14A8882704A88120AC270CA
:107E40000420704702208242FBD14A8804309A7095
:107E50004A88120ADA708A881A718A88120A5A7154
:107E6000EFE710B50400012082420CD94B780A7864
:107E70001B0213432380834206D1CB788A781B02EE
:107E800013436380002010BD022BFBD1CB788A788E
:107E90001B02134363804B790A791B021343A380AF
:107EA000F0E70B8803700B881B0A43704B888370C4
:107EB0004B881B0AC3708B8803718B881B0A437124
:107EC000CB888371CB881B0AC371082070470300DD
:107ED0000120082A14D14A780878120202431A8035
:107EE000CA788878120202435A804A7908791202C5
:107EF00002439A80CA798879120202430020DA800C
:107F0000704710B504000120022A05D100204B78EB
:107F10000A781B021343238010BDF8B50600102019
:107F20000F00150003F034FB04000120002C0ED0DC
:107F3000A0230C22290023806780201D002D07D05C
:107F400003F0BEFB2100300003F0E2F90020F8BD91
:107F500003F06EFAF6E7F7B51E00009008AB1420A8
:107F600017001D78019103F013FB041E12D0A22309
:107F70000370019B47704380099B057146710C2279
:107F80000830002B07D0190003F09AFB210000985D
:107F900003F0BEF9F7BD099903F04AFAF6E737B5E1
:107FA000041E0FD04388002B0CD00025C18813235A
:107FB000007A172201950095FFF7CDFFFF2365801A
:107FC0006372257037BD000010B50C4904004A8863
:107FD000002A09D08B89002B05D00020CB8A0222F1
:107FE000834201D010BD012213000A204343002028
:107FF0004032C854C81842800472F3E7B664FF1FC9
:108000000023438003707047094B00211A0010B50C
:108010005C88002C06D01C79844203D10A234B4390
:10802000D01810BD01310A330329F1D10020F8E73F
:10803000B664FF1F10B50400407A03F0E1F9FF2396
:10804000637210BD7047043010B580B203F0D0FAEF
:10805000002803D00421494203F052F910BD00006A
:1080600070B50025104CA0682580A581A580A84288
:1080700002D003F09DFBA56000250C4C0C4B606DFD
:108080001D80230058331D70A84202D003F090FBDE
:10809000656500256068002801D003F089FB013583
:1080A00008340A2DF6D170BD7C65FF1F2065FF1FC7
:1080B0007065FF1F70B5041E09D1054D2880A88189
:1080C000A880A868002802D003F072FBAC6070BDE5
:1080D0007C65FF1FF0B54B8885B00193002343609A
:1080E0000A7905000F00022A00D07BE0CA88032A23
:1080F00017D98B685E7819783602DC78D8790E4308
:1081000099781B7A24021B020C43034353495BBA40
:108110000B80331D93421ED1042C04D0631F022B0D
:108120000ED9012015E0019A4D4B1201D35A002BB4
:1081300006D00198FFF7BEFF4A4A13690133136165
:108140000421B8682E812C80494203F0D9F8686078
:10815000002005B0F0BD434D042C06D0631F022B58
:108160000FD9EB680133EB60DBE7019A3C4B12015E
:10817000D35A002B05D00198FFF79CFF2B690133E0
:108180002B61374B30000293019B029A1B01019334
:10819000002301998C468B52130063449C80039307
:1081A0009E81FFF750FF039B041E986016D00421A8
:1081B000B868494203F0A4F8FA880100043A2000A4
:1081C00003F07EFA0199029AFB888A5A043B9B18B5
:1081D000029A8B522B6801332B60A2E7AB69013303
:1081E000AB619EE71E4B0293019B1E01029BF35A5B
:1081F000002B2DD002998C19A068002828D0012AC4
:1082000026D1FA889B189BB27352A189994217D341
:108210009B1AC018B96803F053FA029BA289F35A5B
:10822000934200D07DE700222B81A3882B80A36896
:108230006B60029BF2520B4A53680133536070E744
:10824000084A9368013393600198FFF733FF68E7AA
:10825000044A536901335361F6E7C046E664FF1FE1
:108260007C65FF1FEC64FF1F70B5051E15D10B4C1C
:108270000B4B1880230058331870606D002802D013
:1082800003F096FA6565250050356068002801D036
:1082900003F08EFA0834AC42F7D170BD2065FF1FA1
:1082A0007065FF1FF0B51700A12285B09200019301
:1082B0004243394B06001B680C009B18D933FF332F
:1082C0001D78FDF741FF0430854204DD3000FDF7E5
:1082D0003BFF0430C5B2BD4207D33A000021300055
:1082E000019B03F0D5F905B0F0BD2900380003F07B
:1082F00017FA2300C6B250331E700393019B290066
:108300006365380002F0DCFFCBB20293002B02D091
:10831000039B01361E7000262300503303931B7805
:10832000B34204D8606D002831D10020DBE7029A07
:108330002800002A04D0013B1000B34200D02800DE
:10834000F700E719387003F08BFA786000280ED038
:108350003A78019903F0B4F9019A3B780136D318C1
:108360000E4A0193D369F6B20133D361D4E7039B7C
:1083700018706065A74205D1084A1320D36A0133FB
:10838000D362B0E7606803F013FA0834F2E703F051
:108390000FFA00236365C8E73409FF1FEC64FF1F71
:1083A000F7B50D0007000421686802F0A9FF2B89CA
:1083B000040003702B891B0A43702B8883702B8861
:1083C0001B0AC3702E8902250436F6B2F42E15D886
:1083D0001B4B9F4214D10C2003F0DAF81135011E1B
:1083E0000CD0902303708E3B0371043B4380154BEC
:1083F0008460C680187802F08BFF00252800FEBD3F
:108400005C237B43104AD3180093583301931B78A5
:10841000002B0FD10300320038000099FFF742FF14
:10842000019B05001B78002BE8D13800009903F070
:108430005FF9E3E7054A0725536A01335362DDE735
:10844000FEFF0000E464FF1F2065FF1FEC64FF1FB8
:10845000F0B587B0009017200F0016000193FFF7CA
:10846000F2FD1325041E19D00C98031E02D00199A9
:10847000201D9847030AE370052302AAA070043068
:10848000908127700098667003A993800494FFF789
:1084900087FF051E02D0200003F08AF9280007B0EC
:1084A000F0BD0000F0B587B01F000CAB1B78039146
:1084B000059301210DAB06001C78049200F0D6F85C
:1084C0001425002821D02000FFF77EFD0135041E71
:1084D0001BD01149059B0A7803700132D2B2131EDA
:1084E000C68001D101231A000B7022713000049B59
:1084F00003990097FFF7ACFF051E09D12300210067
:108500000648074A093302F0DBFF280007B0F0BD38
:10851000002363802370F8E7E864FF1F9F7F00114A
:1085200030750000F8B505000E00064C064F2368B4
:10853000002B02D03100280098470434BC42F6D109
:10854000F8BDC0468C65FF1FA065FF1F0123064ACA
:108550005B425380002313715362044A13605360DB
:108560009360D36013617047A065FF1F8C65FF1F88
:108570000200002310B506499C000859002801D1CB
:10858000625010BD0133052BF6D11320F9E7C04628
:108590008C65FF1F034A5388181A434258414042D2
:1085A00010407047A065FF1FF0B585B002930AAB7D
:1085B0001F780CAB1B88009008000E0001920393FB
:1085C000FFF7E8FF05001120002D1BD10E48FFF733
:1085D000E1FF04001520002C14D006220B99A7718E
:1085E000E01D03F06DF8019B30002371029B290010
:1085F0006371009B66802370039B6562E381FFF7D4
:1086000091FF280005B0F0BDFFFF000010B5FFF797
:10861000C1FF04000220002C12D060880121FFF766
:1086200081FF606A002801D002F082FE282200212A
:10863000200002F0FDFE012300205B4263802071D8
:1086400010BD000030B5074A074C5588010013786B
:108650000020A54204D05B1A59424B4158421040B9
:1086600030BDC046A065FF1FFFFF0000084A10B5DF
:1086700001230C00904208D0FFF78CFF031E04D0AA
:10868000037923405A1E9341DBB2180010BDC04647
:10869000FEFF0000024B1879431E9841C0B270479C
:1086A000A065FF1F70B504000D001600FFF772FFF4
:1086B000002804D10D4B9C4200D0143070BD416A9B
:1086C00003790520002907D012221A40102A02D16E
:1086D0000520002EF2D10F20DB06EFD5897E0C207D
:1086E000A9428941494249420840E7E7FEFF0000AC
:1086F000030010B5002800D110BD0348034A41888B
:108700009142F9D09847F7E7A065FF1FFFFF0000EF
:10871000002330B5C45CCD5C6C40D4540133102BC5
:10872000F8D130BD0F23002210B5C45C6400224391
:10873000CA54C25CD209013BF7D210BD020001004D
:1087400010B52032103102F03BFF10BDF0B58BB0F8
:108750000390102005931700049102F011FF009080
:10876000102002F00DFF009B13240190002B05D078
:1087700000280CD11324009802F0DAFD019B002B95
:1087800002D0180002F0D4FD20000BB0F0BD102084
:1087900002F0F6FE0600102002F0F2FE132405009F
:1087A000002E00D1AEE0002819D01022002102F0E6
:1087B0003FFE32002900039802F002FF041E0ED192
:1087C00033787F2B51D830000099FFF7ABFF009B27
:1087D0001B787F2B53D801990098FFF7A3FF300037
:1087E00002F0A6FD002D02D0280002F0A1FD002C11
:1087F000C1D1102002F0C4FE0600102002F0C0FE1D
:108800000290002E7CD0002878D03A000F3223004E
:108810000125121105D00F333B4015B25A42534186
:108820001BB26A1E1201002B33D0049BD2B29818DF
:108830000099029AFFF76CFF013D102200213000E1
:1088400002F0F6FDADB2049F2D017D19AF4242D07A
:10885000002C33D0300002F06BFD029B002B00D1C6
:1088600089E7180002F064FD85E729003000FFF772
:1088700059FF28002549009AFFF74AFFA7E729007A
:108880000098FFF74FFF28002049019AFFF740FFAB
:10889000A5E70F210F4004998A18D9B28F4208D951
:1088A000D15C06A819540133102BF6D1029A019914
:1088B000C0E7791A48424141C901F2E73900300066
:1088C00006AAFFF725FF3200039806A902F078FEFA
:1088D00010370400BAE7002CBCD13000029906AA78
:1088E000FFF716FF320006A9039802F069FE08227E
:1088F00004003100059802F0E3FEABE71324A9E77A
:108900001324AAE7002800D06EE733E790BA0011DD
:10891000F0B58BB00F0016000225009000283FD064
:10892000002A3DD00B1DDBB21800029302F028FE96
:108930001135041E34D0FDF747FD05003A000099BB
:10894000201D02F095FCEBB20393E3702B0CDBB21D
:108950002F0A00936370FFB22B0E2370A770019350
:10896000FDF72CFD1022010006A802F081FC210079
:10897000029A04AB06A8FFF7E9FE051E0DD1039B82
:1089800008223370009B04A9B370019B7770F370C9
:10899000301D02F06DFCFDF71DFD200002F0C8FC4B
:1089A00028000BB0F0BDF0B58FB00D00149E039001
:1089B00004920593002A03D1022420000FB0F0BDD9
:1089C000002EF9D00398FFF7E5FD1424071EF4D01C
:1089D0007278337812021A43B3781B041343F27887
:1089E00012061A43036A0192934201D30133E3D181
:1089F000002D03D03B7901249B07DED508220021FE
:108A000006A802F015FD059B13240433DBB2180001
:108A1000029302F0B5FD051ECFD0059A04990430EB
:108A200002F026FC04223100280002F021FC39006B
:108A3000102210310AA802F01BFC2900029A06AB92
:108A40000AA8FFF783FE041E0FD1082206A908A872
:108A500002F00EFC0822311D08A802F0A1FE012838
:108A600007D101990398FDF7C9FC280002F060FCCA
:108A7000A3E70124F9E7000070B51C4C050023684A
:108A8000181E10D0002D14D11A78002A0CD1981C71
:108A9000083202F015FE02F02BFD0135002808D146
:108AA00023681D70012070BD0A331800082202F0EF
:108AB00007FE2368002BF5D0122002F069FD061E88
:108AC0000DD0C1232168037045700231102202309D
:108AD00002F0F6FD23683100587802F019FC206896
:108AE00002F026FC00232360DCE7C046C865FF1FB8
:108AF000F8B504002020FDF755FB0D4EA700BB592B
:108B00000500002B0DD000280BD0D878FF2809D104
:108B100008492A000C55F35907480333611802F03D
:108B2000CFFCF8BD290002F07BFB0028F0D1F8E76C
:108B3000E465FF1FCC65FF1F499D001170B5064D10
:108B400084006359002B05D0D87802F059FCFF222D
:108B50006359DA7070BDC046E465FF1F70B506004A
:108B60008CB00C00150000213022684602F060FC39
:108B700031001022684602F07BFB1D2021000322F9
:108B8000684402F075FB6846FFF7D8FD2D2104000C
:108B900003222800694402F06BFB20000CB070BD7A
:108BA000F0B50700160097B001931CAB1D7830227A
:108BB0001EAB00910AA800211C7802F039FC10229B
:108BC00039000AA802F054FB1022002102A802F08A
:108BD0002FFC0722310002A802F04AFB072202AB59
:108BE0009818631E9C41019902F042FB02AB9C73F2
:108BF0002B005A1E934102AAD3730021102206A80B
:108C000002F016FC06221D9907A802F031FB1A207B
:108C100002ABC01806221F9902F02AFB102200990D
:108C20000EA802F025FB102202AB0EA908781C78D2
:108C3000013A6040D2B2087001330131002AF5D107
:108C40000AA8FFF77BFD102212A904000EA802F06B
:108C500037FD102206AB0EA908781D78013A68404E
:108C6000D2B2087001330131002AF5D10AA8FFF70A
:108C700065FD044310222098E4B212A902F0F8FA2C
:108C8000200017B0F0BD70B50E0014008CB00100CC
:108C9000102268461D0002F0EBFA3100082204A8F9
:108CA00002F0E6FA2100082206A802F0E1FA68467E
:108CB000FFF744FD04001022280008A902F0D8FAAA
:108CC00020000CB070BDF8B506000D000024371967
:108CD000AC4200D3F8BD02F063FC030A3B70631C96
:108CE000DBB201379D4203D90234F054E4B2EEE71F
:108CF0001C00EDE773B506000C000225002819D012
:108D0000002917D0032101A8FFF7DDFF6B469A79F0
:108D10003F231A40013313436A463000937101A97F
:108D20002200FFF71BFF051E04D10322E01C01A94E
:108D300002F0C6FC280076BD03785807DA08C00F99
:108D4000D20080009B0710439B0F1843C0B27047AE
:108D500007230B40C908C9000B430370704700008C
:108D600070B50400FFF7EAFE134DA4006359002B11
:108D700021D0186A002801D002F0DAFA2B59986E37
:108D8000002801D002F0D4FA2B59D86E002801D067
:108D900002F0CEFA2B59186F002801D002F0C8FA61
:108DA0002B59586F002801D002F0C2FA285902F05E
:108DB000BFFA00232B5170BDE465FF1F0E4B8000EE
:108DC000C35870B50C00002B0FD09D68002D0CD03F
:108DD0002B78201D0B706B784B70A97CFFF7B8FFC8
:108DE0002B7E23726B69E36070BD1022002120008E
:108DF00002F01EFBF8E7C046E465FF1F014B186058
:108E00007047C046E065FF1F074A03008000825894
:108E100010B5002A06D0D088984203D1012901D18B
:108E2000FFF79EFF10BDC046E465FF1FF0B5264E5C
:108E300095B087000B93BB590500099112200A9247
:108E4000002B31D0D888FFF7A5FB04001420002C9C
:108E50002AD0280010A9FFF7B1FFBB591E781D6A60
:108E6000002E23D00895FDF7EFFA07000020FDF74C
:108E7000F1FA0790A379E61D069310AD0CA90898A6
:108E800000F0E2FA0EA9280000F0D7FA0B9B0A992D
:108E90000493069B09980293079B039601930097FE
:108EA0000EAB0CAAFFF77CFE15B0F0BDFDF7CCFAB7
:108EB00006903000FDF7CEFAE31DA779079310ABBB
:108EC00006000893DAE7C046E465FF1F30B50C4C96
:108ED00085002A59030085B00120002A0ED0180011
:108EE0006946FFF76BFF2B591A78D888054B002A83
:108EF00000D1054B6A46072100F0D9FB05B030BD13
:108F0000E465FF1F3B9400114994001130B5094CF2
:108F10008500295985B010226846253102F0D0FB22
:108F20002A591121044BD0886A4600F0C0FB05B0D5
:108F300030BDC046E465FF1FE594001130B5094C13
:108F40008500295985B010226846353102F0B8FBFA
:108F50002A591121044BD0886A4600F0A8FB05B0BD
:108F600030BDC046E465FF1F23950011F7B54D4F96
:108F700086001020F4590D0002F002FBF359206224
:108F8000186A132200286CD0033A29009C6802F06A
:108F900097FBF3591A780192002A58D11E6A227D54
:108FA000317B944651400122019F114201D1674615
:108FB0001740217D914339432175377B4F40BC4693
:108FC00060460027800701D44F0817400121022086
:108FD0008F40227D82433A432275377B5740BC46FF
:108FE00060460027400701D497080F400420227DE7
:108FF000BF0082433A432275627D00279446604653
:10900000727B42400A4201D167460F400121627DD6
:109010008A433A436275777B5740BC4660460027D7
:10902000800701D457080F400220627D7F008243F1
:1090300017436775767B00227E40760701D4BA0815
:109040000A400426617D9200B1430A4362756A7842
:10905000002A08D06278002A05D005220533DA7785
:1090600000221000FEBD04222979114205D1A17C05
:10907000114202D10533033AF1E7019A21782C78A5
:10908000002A02D10A002100140018220429E8D87D
:10909000042CE6D805206043034A05331218525CBD
:1090A000DDE7C046E465FF1FA0BA001110B50A0055
:1090B0001121024B00F0FBFA10BDC0467F95001154
:1090C0000B0030B587B001AD2B806B46040011005A
:1090D000981D082202F0F4FA2A000B212000024B0E
:1090E00000F0E5FA07B030BDA795001110B50A00F1
:1090F0001121024B00F0DBFA10BDC046FB950011B8
:1091000013B50B0011006A4613706B46040006226B
:10911000581C02F0D5FA6A4608212000014B00F0E5
:10912000C6FA13BD1B96001110B50A001121024B9F
:1091300000F0BDFA10BDC0466B9600117FB505006A
:109140000B4BAA00D4580800002C0FD0666F237F69
:10915000E28821780396266F0296E66E0196A46E49
:109160000094FDF709FC2800FFF7FAFD7FBDC0461B
:10917000E465FF1F10B51721FFF7E0FF10BD0000E9
:1091800070B50A000D00064B0221040000F08FFAB2
:10919000060029782000FFF7D1FF300070BDC046DF
:1091A0004B95001170B586B000236A461370836832
:1091B00004001D78681E0A2859D801A902F040FA57
:1091C000060633373B3F43474B4F5300180000F030
:1091D00042F9062312284BD000281BD16088FFF7E4
:1091E000D9F90823002813D04279002A47D1264B09
:1091F0001A78072312070BD5244B1A680723002A75
:1092000006D01668002E03D0290001AAB04703003B
:109210006A4613706B461B786088002B2AD1FFF7D3
:1092200067FC06B070BD180000F06CF9D4E71800B8
:1092300000F087F9D0E7180000F093F9CCE71800A8
:1092400000F0ADF9C8E7180000F0C3F9C4E7180052
:1092500000F0F6F9C0E7180000F0F6F9BCE71800D6
:1092600000F013FAB8E7180000F013FAB4E7072388
:109270006A46137069466088FFF782FFD1E70523CD
:10928000012AC5D1024BB8E77164FF1FDC65FF1FDF
:10929000E065FF1FF8B52C4F8600F35904000D0060
:1092A000002B40D0DA8882423DD15A78062A33D149
:1092B0001A78002A2ED0012099681A6A097D014285
:1092C00006D0157B054203D007225A700120F8BD55
:1092D0000220014204D0157B054201D00922F4E7A7
:1092E0000420014204D0127B024201D00B22ECE7A1
:1092F000164B1B68002BE9D05B68002BE6D02000E2
:109300009847BB5900215B78122BDFD12000FFF773
:1093100015FFDBE70E4BECE7112A04D1002900D042
:1093200032252900F2E7002D08D12000FFF732F99D
:10933000002803D010230279134303712100280071
:10934000FDF798FAC2E7C046E465FF1FDC65FF1F22
:10935000E065FF1F70B50E4E8500AB590400002B71
:1093600013D01B78002B11D10A4B1B68002B04D0A3
:109370005B68002B01D02000984773595B78122B53
:1093800003D100212000FFF7D9FE70BD024BECE7AE
:10939000E465FF1FE065FF1FDC65FF1F094B8000D0
:1093A000C3581020002B0CD01A6A002A09D09B68E1
:1093B000002B06D0127A1B7E101C9A4200D9181C72
:1093C000C0B27047E465FF1F70B503000D001400C4
:1093D0000220002A30D000292ED013700B78081DEF
:1093E00053704B789370FFF7A7FCE07001200221C7
:1093F0002B7A23716B7B034063716A7B0A401343B2
:10940000042263716E7B1640334363716E7BF608F2
:10941000F600334363712B7B0340A371287B01402B
:1094200000200B43A371297B0A401343A3712A7BBD
:10943000D208D2001343A37170BD10B50A00010019
:109440000120FFF7C1FF10BD10B50A000100022086
:10945000FFF7BAFF10BD70B506000C000220002E09
:1094600030D000292ED07378201D0B70B3784B704C
:10947000F178FFF76DFC01223579257271794B1077
:1094800008001340934010400343881010408000B0
:10949000C9080343C9000B436373B1794B1008003B
:1094A0001340934010400343881002409200C908C3
:1094B0001343C9000B4321202373FCF773FE85423D
:1094C00001D2122070BD2220257AFCF76BFE854266
:1094D000F7D823781820042BF4D86378012BF1D81F
:1094E0000020EFE7030010B50220002909D0002B6F
:1094F00007D00322481C0A7019000D3202F0E0F870
:10950000002010BD03000222080010B5002B06D079
:10951000002904D00E32591C02F0D2F800221000AB
:1095200010BD030010B50220002909D0002B07D080
:109530000422481C0A7019000C3202F0C1F8002005
:1095400010BD10B5FFF7DEFF10BD0300022000299B
:1095500006D0002B04D0052200200A701B784B7027
:10956000704703000220002B08D0002906D05B784A
:1095700000200B70013B082B00D918307047030006
:1095800010B50220002909D0002B07D00622481C64
:109590000A7019000A3202F093F8002010BD10B5CD
:1095A000FFF7B0FF10BD02000B00022010B500292C
:1095B0000ED0002A0CD0072119701188597011881B
:1095C000090A997011180822D81C02F079F80020B5
:1095D00010BD03000A00022010B5002B0CD000299A
:1095E0000AD099785878090201431180901CD91C3F
:1095F000082202F065F8002010BD030010B502201B
:10960000002909D0002B07D00822481C0A70190035
:10961000921802F055F8002010BD02000B00022045
:1096200010B500290BD0002A09D009211970117832
:1096300018185970511C062202F042F8002010BD83
:1096400010B5FFF75FFF10BD02000B00022010B540
:10965000002A09D0002907D0517819701118062264
:10966000581C02F02DF8002010BD030010B5022098
:10967000002909D0002B07D00A22481C0A701900C3
:10968000063202F01DF8002010BD10B5FFF73AFFBA
:1096900010BD02000B00022010B5002A06D00029E0
:1096A00004D018005178FFF753FB002010BDF0B52F
:1096B00085B017001E006A46062305000800918148
:1096C0009380FEF7C0FC1324011E02900CD03800DA
:1096D000B047041E05D1280001A9FEF76FFA041E49
:1096E00002D0029802F064F82800FFF701FA200087
:1096F00005B0F0BDF0B504008BB00191150000215C
:10970000102202A801F094FE334EA700B859002899
:109710003CD0C388A34239D10378002B36D142789C
:10972000062A18D102000100553235310C3006AB43
:10973000FFF7A9FA002829D12000FFF72FFE020029
:1097400006A902A801F0BCFF200002A901F070FDEB
:1097500001200BB0F0BD816E002917D00B8A112AB1
:1097600028D19D420ED101981231093A02F018F821
:10977000012807D1BB5920009D6EFFF70FFE29007D
:109780000200DEE732212000FFF7D8FC2000FEF7C0
:1097900001FF061E1BD0416A002918D00B8AAB427C
:1097A00015D108220198123101F0FAFF01280ED1DB
:1097B000716A0AE09D42E9D108220198123101F054
:1097C000EFFF0128E2D1BB59996E8A7EB9E72000EC
:1097D00001F0EEFDBCE7C046E465FF1FF0B56B4D40
:1097E00087007E5985B0337802900393002B00D018
:1097F00087E0B368346A01937078062817D1012294
:109800001B7D134202D0217B114218D10222134248
:1098100002D0217B114251D10422134203D0237B79
:10982000134200D08BE0019B5A7DEB5991E0073841
:109830000428F8D801F004FF032E42678300B36EBA
:10984000002B03D11C2001F09BFEB066EB599C6EEF
:10985000002C1CD010220021200001F0E9FD02980C
:10986000FFF79CFD01002000FFF72DFA01F098FEA4
:109870002082200008211230FFF725FA0298FFF716
:109880008DFDA076EB592100D888FFF70FFC082248
:10989000EB591CE0B36E002B05D01A00198AF08832
:1098A0001232FFF70DFC0222019B197DEB59114288
:1098B0003DD0207B10423AD0073208E0F488FCF714
:1098C000DBFD01002000FFF711FC0A22EB595A7062
:1098D000029B9C002A595378073B042B11D8D0884F
:1098E000FEF758FE00284ED0C3895A08D2182849DE
:1098F000029B0298CB542B5941180433254801F0A0
:10990000DFFD05B0F0BDFCF79FFD030001208342A1
:1099100001D100200393EB59DE88FCF79BFD0399EE
:1099200002003000FFF7ECFB019AEB59117D042295
:1099300011420CD0217B114209D00B22C7E7F688D7
:10994000FCF73CFD01003000FFF7EEFB6BE7019AEE
:10995000527D01210A4204D0607B084201D00C22D2
:10996000B5E702210A4204D0607B084201D00E22F2
:10997000ADE704210A4204D0627B0A4201D01022E2
:10998000A5E71222A3E7FA225200B0E7E465FF1F21
:10999000E865FF1F539D001110B5064B1A7804238C
:1099A000100018401A4200D00348FFF727FA0020A1
:1099B00010BDC0467164FF1F3443FF1F70B5040023
:1099C000FFF7D4FA051E43D12000FFF77FFA234E9C
:1099D000A400A0598268937CDB0708D50321036AA1
:1099E0001B790B40012B02D1017F0B430377431DF1
:1099F000D97F8B1E022B0DD8022900D00121C088EF
:109A0000FCF790FF042133591A7F59700A431A77E3
:109A1000280070BD01290CD10223102243700021BF
:109A20000C3001F005FD305910213530FFF74BF9AE
:109A3000EEE70529ECD10223D118437010220C3037
:109A400001F03EFE04233259117F0B431377EAE7FE
:109A500008251828DCD1053DDAE7C046E465FF1F7C
:109A6000F0B58BB0059143887E4F9E00F4591500E8
:109A70000493002C15D1012902D000200BB0F0BDB9
:109A8000101D57781678FFF757F9EB6832000293EC
:109A90002B7A0499019300903B002000FCF70CFF07
:109AA000EBE7E388049A934201D00820E6E72378A5
:109AB000012B00D1D4E0059B581E092800D9CFE026
:109AC00001F0BEFD05CE0A29CC506C859AB2290062
:109AD0000498FFF773FFD1E72000290010224530DA
:109AE00001F0EEFDB9594B78042B02D1013B4B70CC
:109AF000C3E70B000A00253335320C310498FFF719
:109B000095F90498FFF702FA0522431E9841BB59C4
:109B1000C0005A70B2E7200029001022553001F031
:109B2000CFFD049B4F4C9D00295904980A0006ABB9
:109B300055320C31FFF77AF929591022453106A820
:109B400001F02EFE012808D10498FFF7F7F90590DF
:109B5000002804D106222B595A7005988EE7082355
:109B60000593FAE763780C2B7AD1E36E002B03D1CF
:109B70001C2001F005FDE066BB59D86E00286FD0AF
:109B80001022290001F09CFDBB590498DC6EFFF700
:109B900005FC0D22A076BB595A706EE7E06E0028D6
:109BA0005ED063780D2B5BD12B8808220382A91C21
:109BB000123001F085FDBB599A68517D0222114295
:109BC00026D0186A407B104222D00C32E4E763783A
:109BD0000E2B45D1236F002B03D1162001F0D0FCB2
:109BE0002067BB59186F002803D01022290001F00C
:109BF00067FD0F22BB59CFE763780F2B30D1206F61
:109C00000622691C103001F05BFDBB599A68517D3A
:109C10000422114203D0196A497B1142D5D1002197
:109C20000498FFF78BFA28E7636F002B0DD0BB5920
:109C3000586F0028F3D01022290001F041FD0122C5
:109C4000BB5952425B6F1A61E9E7142001F098FC9E
:109C5000BB5960675B6F002BE9D126E72978DFE706
:109C600007200BE7E465FF1F10B5064C207001F0DC
:109C7000FFFB06212078FDF791FF0348FEF778FCF3
:109C800010BDC046F765FF1F098E001100200BB202
:109C900070B50D00834216DA264B187801F070FB80
:109CA000041E0DD00378922B0ED0A02B37D0224B60
:109CB0001878FF283AD0210001F02AFB002835D17E
:109CC00080200002684070BD43780E2B0BD03E2BE5
:109CD000EDD18378052B12D0082BE8D181798088CB
:109CE000FFF7D8FA08E0154B82889A42DFD18368E3
:109CF0001878591CFEF7C0FE002817D1D7E7104B83
:109D00001B785B0712D50F4B1B68002B0ED09B688E
:109D1000002B0BD0C289811D80889847ECE7FFF7A4
:109D200041FAA068002801D001F042FD200001F0B6
:109D30007FFCC5E7F765FF1F2D43FF1F18200000BC
:109D40007164FF1FE065FF1F10B50078FFF712FA7E
:109D500010BD10B50078FFF7FDFA10BD0C2343438A
:109D6000084A10B59B185A68002A03D0012901D16E
:109D7000904710BD9B68002BFBD00029F9D1984774
:109D8000F7E7C0461466FF1F01238340094A10B558
:109D9000946B1C439463506B98435063D46B2000C6
:109DA0009843012901D120001843D063116B0B4364
:109DB000136310BD00800040F0B500240127154B4F
:109DC00085B0DA6B144E03921A6C0192DA64019B2F
:109DD000E3403B4217D0039DE5403D400295E5B28C
:109DE00002992800FFF7BAFF316A736A002908D088
:109DF0003900002B01D0029979402800FFF7C4FFF9
:109E000001E0002BF9D101340C36172CDFD105B05D
:109E1000F0BDC04600800040F865FF1F064B0121E1
:109E20005A68C2400A4204D01B68C3401800084068
:109E300070471B6DF9E7C046008000400122064BC9
:109E40008240002903D0D9680A43DA607047D96894
:109E50009143D960FAE7C0460038004030B503248A
:109E600044430F4BE25C1B199C785D7801232D1B4A
:109E70000135AB40013BA340A140DB430C0012285D
:109E800007D80849920052181168194021431160FF
:109E900030BD054A11680B4023431360F8E7C04604
:109EA000E7BA001108F0004014F00040C21F70B57E
:109EB000D4B20623092C0BD80125084C9540002963
:109EC00008D00021FFF7CAFF23682B43236000233B
:109ED000180070BD2368AB43F8E7C0460038004067
:109EE000214BF0B51B185B78022B21D1032444438E
:109EF0001E4A1F4EA35C121994780122150085405A
:109F0000B76B013CE4B23D43A240B563194C122843
:109F100015D89B0000290CD117495B1899680A4392
:109F20009A600123205C154A834011680B4313603B
:109F3000F0BD11495B18996891439960F1E70E4BA8
:109F400000290DD159690A435A61225C1328E8D0CF
:109F50000123203A93400A49086803430B60E7E76E
:109F6000596991435961F0E7F865FF1FE7BA00119D
:109F7000008000402CBB001100F00040A0F0004029
:109F8000A4F00040F8B500241B4E1C4D1C4B1B5D7B
:109F9000012B1FD1194A9269E2401A420BD00122CB
:109FA000B25693402200143AD2B2022A09D8154977
:109FB0004A6913434B61013402360C35172CE5D145
:109FC000F8BD0022B2560F499200521891680B4317
:109FD0009360F0E7022BEED1E7B23800FFF71EFFE7
:109FE00001235840C1B23800FFF77AFF3800FFF76D
:109FF00015FF6877DFE7C046B9BA0011F865FF1FA3
:10A00000F965FF1F00F00040012202388240054B35
:10A01000002903D059690A435A617047596991432D
:10A020005961FAE700380040F8B50E0001210F0031
:10A030008740114A0400D368FD43BB43D360831EAD
:10A040008B4201D8FFF7E0FF00212000FFF72EFF31
:10A050000A4A0B4B5168012E05D139431B19516037
:10A060005E700020F8BD2940516002221C19627008
:10A070009A6915409D61F4E7003800400080004077
:10A08000F865FF1F012210B58240074B002906D05A
:10A0900019680A431A600121FFF7C6FF10BD19684D
:10A0A00091431960F7E7C046008000400C2370B56B
:10A0B000002543430A4A29009B181D70094B0400E0
:10A0C0001B185D70FFF7B0FF0123A340064928006D
:10A0D0000A681A430A6005490A689A430A6070BD13
:10A0E0001466FF1FF865FF1F348000403080004079
:10A0F00070B504000E00FF2813D003250540FFF7BC
:10A10000D5FF084AA3089B009B183F22ED00AA40F8
:10A11000AE40196820009143314319600121FFF7D7
:10A120008DFE70BD18380040F8B50C244443134B25
:10A130000500E4186368002B03D1A3681220002BEC
:10A140001AD0022201270E4B00215B195A702800F9
:10A150002770FFF769FF63681E1E08D0A3683E00E2
:10A16000002B04D02800FFF759FE4640F6B2280025
:10A170003100FFF709FE0020F8BDC0461466FF1F3E
:10A18000F865FF1FF7B5C420FF222B4B800019583C
:10A19000002491433F3A0A431A508022274F52022B
:10A1A000274E1A60274B1D5D002D21D0A31E012BC9
:10A1B00003D80121E0B2FFF727FF012D18D11F4B73
:10A1C0009B69E3402B4213D0E3B218000193FFF7E1
:10A1D00025FE01000198FFF755FFE3B2143B022B67
:10A1E0001DD801217156184A8D405369AB43536104
:10A1F0003B7F002B0DD0E5B22800FFF795FF28002C
:10A20000FFF70CFE7B7F0100834202D02800FFF79E
:10A21000A5FD01340C370236172CC3D1F7BD01213F
:10A2200000237156F3568D40074A9B009B189A688D
:10A23000AA439A60DCE7C04600E100E0F865FF1F32
:10A24000B9BA0011F965FF1F00F0004010B50121F7
:10A250000400FFF7E9FE0123044A002011194B70A6
:10A26000A34091690B43936110BDC046F865FF1F81
:10A2700070B50E0015000400FFF718FF0C236343B0
:10A28000094A20009B189D605E60FFF74DFFF0219A
:10A29000064B074A8900051E5A5002D02000FFF7DE
:10A2A00005FF280070BDC0461466FF1F0000FF1F99
:10A2B000B99D001170B5134D07202C78002C1FD1CB
:10A2C000982221005200280001F0E2F80123C42066
:10A2D000FF222B700C4B80001C635C630B4B1C60DB
:10A2E0005C600B4B195891433F3A0A431A50802245
:10A2F00052021A600D20074A074901F091F8200028
:10A3000070BDC046F865FF1F00800040A0F000400F
:10A3100000E100E085A10011859F0011030010B548
:10A320000620072B09D8054A137001F091F8D721B0
:10A330000020034B034A89005A5010BD5C43FF1FA5
:10A340000000FF1FD91AFF1F70B51D0002240C2941
:10A3500010D8094ACA40D2070CD5FBF72FFF041EBC
:10A3600008D1059A04992800FBF744FFFCF7B2FDD9
:10A37000FFF712FB200070BD1210000030B50D7801
:10A3800002232C009C43184201D02B431C000825BB
:10A390002300AB43284201D02B00234320241D007F
:10A3A000A543204201D01C4325002A230D701842EA
:10A3B00004D011781E3B0B43137030BD0028FCD134
:10A3C0000C2113788B43F7E7F8B51D0006AB1B880B
:10A3D000140007AA0E000B201778002B27D10A784B
:10A3E000022A49D14A68507811780002244A084369
:10A3F0008018042840D801F023F903121D1B230004
:10A40000F06801F03DF9021CC0B2B84200D93A1C14
:10A41000D2B22000F1682A8001F052F906E002224F
:10A42000F3681B882A8023701B0A63700020F8BD24
:10A430000622EEE701232B80F3681B782370F5E7F3
:10A44000F368002B16D008222A801A8822701A88F6
:10A45000120A62705A88A2705A88120AE2709A88A8
:10A4600022719A88120A6271DA88A271DB881B0A4B
:10A47000E371DBE72B80D9E701202B80D7E7C046CB
:10A4800000D6FFFFF7B516000A781D0008AB1F883D
:10A490000C000123022A18D14A6850781178000272
:10A4A0002B4A0843801803280FD801F0C9F8022569
:10A4B0004439E06801F0E4F8C0B20723B84204D39D
:10A4C0007B190193152B02DD0D231800FEBDE068FA
:10A4D0002A003100C01901F0F3F86B4600209B8878
:10A4E000E268D0541B4B1B68834203D01B68834235
:10A4F00000D098470023E8E70B23002FE5D1022D79
:10A50000E2D1737832781B021343E2681380114B57
:10A510001B68002BEED01B68002BEBD00120E8E776
:10A520000B23002FD1D1062DCED12A003100E068B7
:10A5300001F0C6F8DEE70B23002FC6D1012DC3D1F1
:10A5400032787533012AC0D8E3681A70D2E7C04662
:10A5500000D6FFFF0468FF1F70B50C001500072828
:10A5600037D801F06DF8041436361B36242E182027
:10A5700015290BD8184E16220021300000F058FF84
:10A5800022002900300001F09BF8002070BD182047
:10A590000229FBD11288114B1A80F6E718200829EE
:10A5A000F4D10A000E48290001F0B2F8EDE71820B6
:10A5B0000129EBD10B4B10780B49DA69FFF7DEFE6E
:10A5C000E3E718200129E1D1064B10780749DA6B3F
:10A5D000F4E70220DAE7C046EC67FF1FDA43FF1F0B
:10A5E000D043FF1F6043FF1F8843FF1FA843FF1F87
:10A5F000030010B50020DB0704D50721024A0348F9
:10A6000000F08CF810BDC04644BB00116043FF1F32
:10A61000054A03001068002803D082889A4201D1BD
:10A62000806870470068F6E7FC69FF1F0A8803002E
:10A6300008009A4204D08A8804309A4200D0002050
:10A6400070470000F8B5F22200230D4F0D4E7968D7
:10A65000050042433370994200D07B600A4C0021D0
:10A66000200000F0E5FE00231A007C60AB4202D11E
:10A6700000203370F8BD01332280DBB2F234F5E7FD
:10A68000F46AFF1FF26AFF1F006AFF1F73B56B4673
:10A6900001900600684615001980FCF74DFF041E66
:10A6A00011D1002D0FD07689002E11D00C2000F092
:10A6B00067FF00280ED0084A046013688680856012
:10A6C000002B02D11060200076BD1A001B68F7E74E
:10A6D0000224F8E71324F6E7FC69FF1F012100229A
:10A6E0000A4B10B549420A4C198099809A719A70A8
:10A6F000084B2070012019805A60FFF7A3FF2078D3
:10A70000FCF778FF0448FDF733FF10BD0C68FF1F0E
:10A71000FC6AFF1FF46AFF1FC9A70011022310B5CE
:10A72000002802D0FFF7B2FF0300180010BD0000A0
:10A73000030010B50020DB0704D50421024A0348BA
:10A74000FFF7A4FF10BDC04658BB0011E043FF1F38
:10A75000F0B50E2687B003930CAB1F8802ABF6183A
:10A760000500080031000292FDF768F8040001209E
:10A77000002C0FD03088FFF74BFF03000E20002B7A
:10A7800008D05E68002E05D021002800039B029AA5
:10A790000097B04707B0F0BD0A4B10B5984207D1FB
:10A7A0000122002352420A808B708A808B7110BD77
:10A7B000FFF73CFF0028FAD001235B42038000230F
:10A7C0008370F4E7FFFF0000F8B5050001290AD106
:10A7D000134E00243388F227AB4219D028001149C8
:10A7E000FFF7DAFF06E0022904D10139FDF73EFF49
:10A7F0000028EDD0F8BD3B0063437268D018D35AEF
:10A80000002B09D03A00002100F012FE0134E4B21E
:10A81000054B1B78A342EED801235B423380DDE772
:10A82000F46AFF1F0C68FF1FF26AFF1F10B5FFF7E5
:10A83000FDFE03000020834200D0987810BD000088
:10A84000F0B589B01C000EAB80CB03901E8810AB16
:10A850001B78049202930B7A0D00DB0616D42B783A
:10A860000593022B24D00498FFF7D2FE002812D0C3
:10A8700003689C46002B0ED0029B22000193290006
:10A880003B00644603980096A04705E00498FFF754
:10A89000BFFE002802D10E2009B0F0BD8368002B56
:10A8A000F9D00A222900039898470028D7D0F3E767
:10A8B0006B6858781A786B4B000210439842D2D8D4
:10A8C000043B984210D2684B984242D015D8674B4F
:10A8D000C0180128C7D80B20002EDDD1EB681A78EC
:10A8E00059683A80200028E0614BC018032800D93D
:10A8F00079E000F0A5FE846A789E5E4B9842B2D162
:10A900000B20002EC8D101233B80EB6831001B785F
:10A9100023706889013080B2FCF790FF3A88031EEB
:10A920000ED0017802328A183A80428962704289D8
:10A93000120AA27059680278E01C00F0C1FE06E01D
:10A9400004323A8031000422601C00F071FD0020C6
:10A95000A2E70B20002E9FD1EB6807A91E880423D5
:10A960003B80330A300026706370FCF767FF051EDA
:10A9700028D004AB9A890E2304A95B183E49C66807
:10A98000FCF7D0FF00280BD12B783C486A6805996A
:10A99000FBF786FB002803D1012304AA5B42D38185
:10A9A0003278022A06D17168201D00F089FE3B88AA
:10A9B00002333B800E2304AA9B181B88A3701B0A3A
:10A9C000E370C4E704ABDE81F4E70B20002E00D077
:10A9D00062E7E9680398FFF729FF02233B802070B4
:10A9E000000A6070B3E70B20002E00D054E702226B
:10A9F000EB681B883A8023701B0A6370A7E7E8683E
:10AA000000F03EFEC2B203000720B24200D243E78C
:10AA10000DD00299DBB27118994202DB921BD3B2BE
:10AA20000293029BE9681A003B8089195AE70023C8
:10AA3000F6E70B20002E00D02EE70722EB683A80C5
:10AA40001A7822705A7862705A88A2705A88120A4C
:10AA5000E2701A792271DA886271DB881B0AA371AD
:10AA600075E7C046042900000228000000D8FFFF57
:10AA7000FFD6FFFF03280000FFFF000088BA001187
:10AA8000F0B58DB06B460020089120229B5E83427A
:10AA90003DDAA64B187800F073FC071E32D003781D
:10AAA000B02B2CD10079023816281FD800F050FEA8
:10AAB00017001E001E001E0031001E0096001E0022
:10AAC0001D011E0052011E0073011E00CD011E005B
:10AAD00050021E001E001E008E021E00E302944B58
:10AAE00094491B8878880B80FBF71AF83800FCF72C
:10AAF0009BFF914B1B68002B01D038009847380012
:10AB000000F096FD8020089B0002434018000DB025
:10AB1000F0BDEE220021874800F08AFC0BAA3B7BA7
:10AB20007989388900923A000D32FCF79FFD0400C4
:10AB3000804B1B78002C3FD146E0804B78880593F2
:10AB40007F4B4100CB5A0BAE073BDBB232880293FE
:10AB5000002301937B4B210006930093059BFFF795
:10AB60006FFE744D002810D1069B3A8A1B889A42CA
:10AB70000BD138000599123000F012FE002804D0E5
:10AB80002B7862899B00EB185A80162306A81B18A5
:10AB9000328820007989FCF7C5FE2B7804009A00E2
:10ABA000AA1851880029C3D00133DBB22B700028CA
:10ABB00007D006A9C98A9180634A12889A42BCD8F4
:10ABC00002E0012149429180002B04D05949788844
:10ABD000FAF7DAFF8AE73E890A2479E000253E8900
:10ABE000574B06937B88069A5B009B5A033B9D421A
:10ABF00002DB002DF0D05BE0162206A812183B7B8A
:10AC0000798900923A0030000D32FCF72FFD059053
:10AC1000002858D04689017A7888FCF7F1FC041E98
:10AC200044D1464B78880793069B4100C95A454B4F
:10AC30000439C9B206AAD28A0693029101940093FC
:10AC40000599079BFFF7FCFD041E2FD1069B394990
:10AC50001A88931C002D26D14B807988384B4900E7
:10AC6000CB5A5119033B8B4220DD059B31485B8950
:10AC700041190B71A91C0135C9B2EDB205914519F5
:10AC80001B0A2B71059B2D490433181800F018FD81
:10AC90002C4B059A1B88D318DDB22C4B9E4205D055
:10ACA0000136B6B29CE749889942D6D0002D0CD027
:10ACB000204C2800618800F083FB207021007888F8
:10ACC000FAF772FF12E7059CF0E7002C00D183E74A
:10ACD0007B78142B00D109E716493B794E800B7025
:10ACE0000C717888FAF712FF00E7162406ABE41817
:10ACF00021003889FCF7A2FD011E00D1B7E1788858
:10AD000022880F4C45002C5B0A4D013CE4B20294B2
:10AD100000240F4B01940095FFF792FD041E00D014
:10AD200014E129007888FAF74FFFDFE6FC6AFF1F7D
:10AD3000CC42FF1F1468FF1F0868FF1F0869FF1F30
:10AD40004464FF1FF869FF1FCA42FF1FFFFF000096
:10AD50001668FF1F162406ABE41821003889FCF79B
:10AD60006DFD011E00D182E178882288AE4C45003D
:10AD70002C5BAE4D013CE4B202947C89AC4B019457
:10AD80000095FFF75DFD041E00D0DFE02900788804
:10AD9000FAF724FFAAE60025A44B1D803B00F633FA
:10ADA0001B78A24A78880792AB4208D99E4B12883A
:10ADB0000693069943005B5A013B9A4203DB0799CD
:10ADC000FAF716FF92E616246B00FB18059306AB04
:10ADD000E418059B21001889FCF730FD011E03D102
:10ADE000059B01241E8973E77888924B2288069C74
:10ADF000099343001B5B904E013BDBB2029300239F
:10AE000000960193099BFFF71BFD041E02D0059BD2
:10AE10001E895DE77B88069A5B009B5A079A10881B
:10AE200032881218934202DC1B1A013B33807F4C9C
:10AE3000023032880999001900F042FC23883288D8
:10AE400001359B182380EDB2A8E70BAA3B7B7989DB
:10AE5000388900923A000D32FCF708FC0025059075
:10AE6000059B002B04D10A24002D00D16EE060E088
:10AE7000059B7888197AFCF7C3FB0100041E63D197
:10AE8000694C6C4B788806940993069B4400E45AFD
:10AE9000694B063CE4B20BAE3288079302940191F1
:10AEA00000930599099BFFF7CBFC041E4CD1079B2F
:10AEB0005E491B881A1D002D30D14A80059B5B4CD2
:10AEC0005A8963191A716B1C9BB2E318120A1A7122
:10AED000162306A832881B1879890598FCF722FDED
:10AEE000FF21AA1C2E1D03350B00059092B2B6B2AD
:10AEF000ADB2002803D006ABDB8AD9B21B0AA21878
:10AF0000651911712B714C4D301D2A884949201843
:10AF100000F0D6FB2B88F618B5B2A1E7498891421C
:10AF200007D17A8806995200525AEB18053A9A428C
:10AF3000C4DC3E4C2800618800F0F2FB2070210048
:10AF40007888FAF75FFED1E5002DF2D13E89BFE6A1
:10AF5000162606ABF61831003889FCF76FFC3D0069
:10AF60000400FA3500282DD0037A9B060CD4002269
:10AF70007B893989788800923A000C32FFF7E8FB28
:10AF8000041E10D03E8915E03088FFF741FB0028F1
:10AF90001AD08368002B17D0210012227888984796
:10AFA000041EE4D0EEE72B78002B02D17888FAF764
:10AFB00039FE00262B78002B00D097E5002C00D11D
:10AFC00094E585E60124DDE70E24DBE7162506ABD4
:10AFD000ED1829003889FCF731FC041E47D0037AAC
:10AFE0009B0611D4154A7B881188994203D01448D6
:10AFF000814207D11380134BF2261D780023D9B26A
:10B00000A94221D30924A1E72888FFF701FB0028E2
:10B010002FD08368002B2CD02100122278889847EB
:10B02000041EDFD092E7C0464464FF1F1468FF1F70
:10B030001668FF1F0869FF1FF869FF1FF46AFF1FEA
:10B04000FFFF0000F26AFF1F3100594354680133CB
:10B050006018615A0029D2D13C0008342100F22244
:10B0600000F02EFB21007888FAF7E4FD3EE501248C
:10B070006CE70E246AE71D4B1A887B889A4231D010
:10B080007888FAF7E1FD31E5F223059851684343EA
:10B09000CD18C95A00291FD03B7A012B0BD16C88DF
:10B0A000AB887888AA1D0094FFF752FB041E02D0DB
:10B0B00000233B722E88F2220021280000F0B8F90C
:10B0C00000232B80059B0133DBB20593084B0599C8
:10B0D0001B78064A8B42D7D801235B421380002C91
:10B0E000CED0F5E5002634000596EFE7F46AFF1FA1
:10B0F000F26AFF1F70B504000E001500FFF796FA04
:10B10000031E08D131000548FFF790FA0300112013
:10B11000002B02D01C8000209D7070BDFFFF00003E
:10B12000F8B50B4F06003B780D001400FF2B0ED036
:10B130000A2000F02DFA011E09D0B123038000235C
:10B1400046800371C5800481387800F0E1F8F8BDCD
:10B150002144FF1FF7B50F0008A90600088809A9B8
:10B160000B240988002821D10234022B1ED15578E6
:10B1700013782D021D432B008B4301937334002B56
:10B1800014D1FB68300019000093FFF74FFB019CBE
:10B1900085420BD02A0030000099FFF7ABFF041E58
:10B1A00004D12A0030007989FFF7BAFF2000FEBDE4
:10B1B000F0B50E7885B003900AA805880120022E0C
:10B1C0000DD14C682778647824023C43054FBC427B
:10B1D00005D10398DBB201960095FFF7BBFF05B0E0
:10B1E000F0BDC04602290000034B10B51B68002BC0
:10B1F00000D09847FEE7C046006BFF1F07B501A8C7
:10B20000FFF7F2FF044A05480021121A00F040F946
:10B21000F8F7F0FAFEE7C046046BFF1F2444FF1F57
:10B2200001B40248844601BC604700BF5147010099
:10B2300001B40248844601BC604700BF311B0000D6
:10B2400001B40248844601BC604700BF193BFF1FA0
:10B2500001B40248844601BC604700BF193AFF1F91
:10B2600001B40248844601BC604700BFC51D000010
:10B2700001B40248844601BC604700BF455101004B
:10B2800001B40248844601BC604700BF1D4B010069
:10B2900001B40248844601BC604700BF8538FF1FE7
:10B2A00001B40248844601BC604700BF456B010001
:10B2B00001B40248844601BC604700BFC52DFF1F92
:10B2C00001B40248844601BC604700BF090E00007B
:10B2D00001B40248844601BC604700BF79180000F1
:10B2E00001B40248844601BC604700BF792DFF1FAE
:10B2F00001B40248844601BC604700BF691F0000DA
:10B3000001B40248844601BC604700BF55490100B2
:10B3100001B40248844601BC604700BF594F010098
:10B3200001B40248844601BC604700BFC52100004B
:10B3300001B40248844601BC604700BF014C0100D3
:10B3400001B40248844601BC604700BF657101003A
:10B3500001B40248844601BC604700BF6DBC0000D8
:10B3600001B40248844601BC604700BF8D12000052
:10B3700001B40248844601BC604700BF0132FF1F90
:10B3800001B40248844601BC604700BFF54E01008D
:10B3900001B40248844601BC604700BFD92FFF1F9B
:10B3A00001B40248844601BC604700BFC94A01009D
:10B3B00001B40248844601BC604700BF091B00007D
:10B3C00001B40248844601BC604700BF350E00004E
:10B3D00001B40248844601BC604700BF4D38FF1FDE
:10B3E00001B40248844601BC604700BF5D170000FD
:10B3F00001B40248844601BC604700BFA54F01006C
:10B4000001B40248844601BC604700BF11470100F7
:10B4100001B40248844601BC604700BF5952010094
:10B4200001B40248844601BC604700BF6130FF1F81
:10B4300001B40248844601BC604700BF154D0100BD
:10B4400001B40248844601BC604700BFC9A900009E
:10B4500001B40248844601BC604700BFD91AFF1FEF
:10B4600001B40248844601BC604700BF4537FF1F56
:10B4700001B40248844601BC604700BFC9260000F1
:10B4800001B40248844601BC604700BFC538FF1FB5
:10B4900001B40248844601BC604700BFB70E0000FB
:10B4A00001B40248844601BC604700BF1930FF1F49
:10B4B00001B40248844601BC604700BF055E00003D
:10B4C00001B40248844601BC604700BFA9460100A0
:10B4D00001B40248844601BC604700BF75A9000062
:10B4E00001B40248844601BC604700BF2526000025
:10B4F00001B40248844601BC604700BFD91B00006C
:10B5000001B40248844601BC604700BF21460100E7
:10B5100001B40248844601BC604700BF5933FF1F95
:10B5200001B40248844601BC604700BF9135FF1F4B
:10B5300001B40248844601BC604700BFC56D0100EC
:10B5400001B40248844601BC604700BFADAE0000B4
:10B5500001B40248844601BC604700BF3D180000AA
:10B5600001B40248844601BC604700BFB14E0000F0
:10B5700001B40248844601BC604700BFE1170000E7
:10B5800001B40248844601BC604700BF3D4B010046
:10B5900001B40248844601BC604700BF1D4D010054
:10B5A00001B40248844601BC604700BF2951010034
:10B5B00001B40248844601BC604700BF9D35FF1FAF
:10B5C00001B40248844601BC604700BFE548000062
:10B5D00001B40248844601BC604700BF7139FF1FB7
:10B5E00001B40248844601BC604700BFB54C01006D
:10B5F00001B40248844601BC604700BFE92800004E
:10B6000001B40248844601BC604700BFED4A010016
:10B6100001B40248844601BC604700BFF94C0100F8
:10B6200001B40248844601BC604700BF51250000B8
:10B6300001B40248844601BC604700BF434D01008D
:10B6400001B40248844601BC604700BF2D3BFF1F88
:10B6500001B40248844601BC604700BFF30E0000FD
:10B6600001B40248844601BC604700BF2932FF1F75
:10B6700001B40248844601BC604700BF0D5201007E
:10B6800001B40248844601BC604700BFDD5201009E
:10B6900001B40248844601BC604700BF5118FF1F37
:10B6A00001B40248844601BC604700BF851F00000A
:10B6B00001B40248844601BC604700BF4D1F000032
:10B6C00001B40248844601BC604700BFE94C010058
:10B6D00001B40248844601BC604700BF85520100A6
:10B6E00001B40248844601BC604700BF45500000D9
:10B6F00001B40248844601BC604700BF7D18FF1FAB
:10B7000001B40248844601BC604700BF291C000008
:10B7100001B40248844601BC604700BF810E0000AE
:10B7200001B40248844601BC604700BF090E000016
:10B7300001B40248844601BC604700BFC12FFF1F0F
:10B7400001B40248844601BC604700BF9DA90000C7
:10B7500001B40248844601BC604700BF413BFF1F63
:10B7600001B40248844601BC604700BFB3520100E7
:10B7700001B40248844601BC604700BF01240000B8
:10B7800001B40248844601BC604700BFEDA500003B
:10B7900001B40248844601BC604700BF156B01003C
:10B7A00001B40248844601BC604700BFCD4C010093
:10B7B00001B40248844601BC604700BFD94901007A
:10B7C00001B40248844601BC604700BF2124000048
:10B7D00001B40248844601BC604700BF35550000F3
:10B7E00001B40248844601BC604700BFDD66010029
:10B7F00001B40248844601BC604700BF8B5201007F
:10B8000001B40248844601BC604700BFED39FF1F08
:10B8100001B40248844601BC604700BF9136FF1F57
:10B8200001B40248844601BC604700BFC135FF1F18
:10B8300001B40248844601BC604700BF55220000A5
:10B8400001B40248844601BC604700BF0539FF1FB0
:10B8500001B40248844601BC604700BF3938FF1F6D
:10B8600001B40248844601BC604700BF017F00006C
:10B8700001B40248844601BC604700BF056A00006D
:10B880000001010302030303040305020602070289
:10B89000080209000A030B030C020D000E030F033C
:10B8A000100311031303140315001600CD3B001100
:10B8B000013C00110000000002000000C2B80011AD
:10B8C000192A0F180A000000F1590000FD24000099
:10B8D00041460100797C00118D9C0011E17000113E
:10B8E0007D7A00118D52001181AA0011014F0011C3
:10B8F000DD3D00110D3F0011000000001616000094
:10B90000020000000CB90011F4FFF3FFD2FC0000AC
:10B910004D400011000000000000000054757961E6
:10B920000042312E3500303031340067697468755B
:10B93000622E636F6D2F70767678004254483031F6
:10B94000000000000200000058B90011292A282A2E
:10B95000272A262A252A242A0A180000E2040000A1
:10B960007102000078EC0000744000001027000015
:10B9700060F0000006640000204E0000000000009F
:10B98000050000001F501D00023CB400000114001F
:10B990001500000081020000303132333435363773
:10B9A0003839414243444546000000009156001199
:10B9B000E55600110000000002000000C4B90011AB
:10B9C0006F2A6E2A1A18000001A000000000000073
:10B9D0006410B71DC8206E3BAC30D9269041DC7690
:10B9E000F4516B6B5861B24D3C7105502083B8ED3A
:10B9F00044930FF0E8A3D6D68CB361CBB0C2649B5E
:10BA0000D4D2D38678E20AA01CF2BDBDFB349B5F82
:10BA1000800000800010000000000000E35C0011C6
:10BA20006D730011075D0011757700118B5D0011BA
:10BA30004B770011015E001121770011535E001158
:10BA4000E9780011BB5E0011E9780011ED5E00118C
:10BA5000A3780011015E0011D9760011795E001102
:10BA60008178001100000000000000005F5F0011FD
:10BA700081780011C15F001185730011052A042A25
:10BA8000012A002A02290328012800280118001889
:10BA9000000000000000000000000000000000871F
:10BAA0000101020102010102010203030401030179
:10BAB000010101010303020103000D000E0010004B
:10BAC000110013001401070108010A010B011C01F8
:10BAD0001D02040205020702080219021A021C02D2
:10BAE0001D030103020317000201000504000807FB
:10BAF000000B0A001716001D1C01020101050401BC
:10BB00000E0D011110011413011716011A1902026A
:10BB100001020B0A020E0D02111002141302171675
:10BB2000030504030807030B0A030E0D00010203BB
:10BB300007090A0B0E0F101112141718191A1B1FE0
:10BB400020212200C9A3001185A4001100000000DB
:10BB5000020000008EBA001100000000B1B1001117
:0CBB600000000000020000008CBA001180
:020000041FFFDC
:1000000000000000453D0011C8B80011C4B800113F
:100010003061FF1F00000000000000000000000031
:1000200000000000000000000000000000000000D0
:1000300000000000000000000000000000000000C0
:1000400000000000000000000000000000000000B0
:1000500000000000000000000000000000000000A0
:100060000000000000000000000000000000000090
:100070000000000000000000000000000000000080
:100080000000000000000000000000000000000070
:100090000000000000000000000000000000000060
:1000A0000000000000000000000000000000000050
:1000B0000000000000000000000000000000000040
:1000C0000000000000000000000000000000000030
:1000D0000000000000000000000000000000000020
:1000E0000000000000000000000000000000000010
:1000F0000000000000000000000000000000000000
:1001000000000000000000000000000000000000EF
:1001100000000000000000000000000000000000DF
:1001200000000000000000000000000000000000CF
:1001300000000000000000000000000000000000BF
:1001400000000000000000000000000000000000AF
:10015000000000000000000000000000000000009F
:10016000000000000000000000000000000000008F
:10017000000000000000000000000000000000007F
:10018000000000000000000000000000000000006F
:100190004D32FF1FAD30FF1FC1660100000000009F
:1001A000000000000000000000000000000000004F
:1001B000000000000000000000000000000000003F
:1001C000000000000000000000000000000000002F
:1001D000000000000000000000000000000000001F
:1001E000000000000000000000000000000000000F
:1001F00000000000000000000000000000000000FF
:1002000000000000000000000000000000000000EE
:1002100000000000000000000000000000000000DE
:1002200000000000000000000000000000000000CE
:1002300000000000000000000000000000000000BE
:1002400000000000000000000000000000000000AE
:10025000000000000000000000000000000000009E
:10026000000000000000000000000000000000008E
:10027000000000000000000000000000000000007E
:10028000000000000000000000000000000000006E
:10029000000000000000000000000000000000005E
:1002A000000000000000000000000000000000004E
:1002B000000000000000000000000000000000003E
:1002C000000000000000000000000000000000002E
:1002D000000000000000000000000000000000001E
:1002E000000000000000000000000000000000000E
:1002F00000000000000000000000000000000000FE
:1003000000000000000000000000000000000000ED
:1003100000000000000000000000000000000000DD
:1003200000000000000000000000000000000000CD
:1003300000000000000000000000000000000000BD
:1003400000000000000000000000000000000000AD
:10035000000000000000000000000000000000009D
:10036000000000000000000000000000000000008D
:10037000FDB10011000000000000000000000000BE
:10038000000000000000000000000000000000006D
:10039000000000000000000000000000000000005D
:1003A000000000000000000000000000591AFF1FBC
:1003B000000000000000000000000000000000003D
:1003C000000000000000000000000000000000002D
:1003D000000000000000000000000000000000001D
:1003E000000000000000000000000000000000000D
:1003F00000000000000000000000000000000000FD
:08183800106FFF1F4118FF1F94
:10184000024981F3088802F06FFA0000106FFF1F51
:1018500010B502F089FA072804D0122808D002280F
:1018600008D010BD044A0420136B01331363F8E75A
:101870000220F6E71420F4E7EC64FF1FF8B5070038
:101880000C0026002500503630785135002804D150
:101890000300287058342370F8BD2978CA00481E08
:1018A0008141A3183800A25C5B68C9B2FFF7D0FF82
:1018B00000280DD12B78DA00A218013350602B706C
:1018C0003378044A013B3370136A01331362D8E75B
:1018D0000123DFE7EC64FF1F5C234343074910B596
:1018E000C9180B0058331B78012B05D1FFF7C6FF31
:1018F000034A936A0133936210BDC0462065FF1FFF
:10190000EC64FF1F10B502F037FB064A01211300FB
:1019100010CB4942D967044B136002F0E5F920006F
:1019200010BDC04600E100E01000100010B504003A
:1019300002F022FB024B1C6002F0D6F910BDC0463B
:1019400000E100E0431E5A425341A022F0B5D2010B
:101950005B421340154D164A40019B182A18127E0F
:101960008BB00191002A1BD01A000832D46F0022DC
:10197000E6B206AFE4B294420EDC2818C369002B2D
:1019800008D0019902AA117106AA049202AA16733C
:1019900003A898470BB0F0BD1978B9540132EAE7B3
:1019A0001A7D1A7806AB01261A70E6E7AC67FF1FAE
:1019B00000400040F0B5254B04004001C25C85B0FA
:1019C000002A2BD01A18117E002927D0917E0029D9
:1019D00024D01179022921D11689D788D168F51B25
:1019E000ADB22A1C102D00D9102292B2BE4217D1DE
:1019F0001818012303710023C269C38003819A422E
:101A000006D06846032103730171029301A8904731
:101A10000820002C00D0192001F0FEFA05B0F0BD1E
:101A2000013C65426C41A0256442ED012C40084D0B
:101A30001B186419074D0633013A92B2AA42EDD041
:101A40001888461C1E80085C2070F5E7AC67FF1FF5
:101A500000400040FFFF00000F220E4B10B59868B9
:101A6000104002380A280BD802F060F80D0A0B0A61
:101A70000A110A0A0A0A060002210020FFF762FF83
:101A800010BD0121F9E70020FFF794FFF8E7DB6FB5
:101A9000F6E7C046004000400F220E4B10B5986894
:101AA000104002380A280BD802F040F80E0A0B0A40
:101AB0000A120A0A0A0A060002210120FFF742FF61
:101AC00010BD01210800F9E70120FFF773FFF7E7D8
:101AD000DB6FF5E70090004013B5334C2378072BFC
:101AE0003DD8324B1A78324B002A39D180221968FE
:101AF00052020A431A60252001F0C4FE20232D4A19
:101B000011680B43802113606B460422C9050868E5
:101B10000733104228D080210422C905C86810422A
:101B20002ED080212020C905CA688243CA601422B1
:101B30001A701A78002A2FD18021C905C86820326E
:101B40000243CA6014221A701A78002A28D11A4B4C
:101B50001A7D22785A601D221A705932DA6013BD3C
:101B60001A6816490A40C5E7086802430A60142249
:101B70001A701A78002ACED01A78013AD2B2F7E752
:101B8000C8680243CA6014221A7019784A1ED2B279
:101B90001A700029F9D1C4E71A78013AD2B2C7E71E
:101BA0001A78013AD2B2CEE75C43FF1F2444FF1FEC
:101BB0003CF000405443FF1F00200040FFFFFEFFA9
:101BC000564B70B51B68012B03D1554A936D0133F9
:101BD000936502F011F9534B534A1860534B544C20
:101BE0001A600123534A1360534A13602378002B71
:101BF00006D006225149524802F0A6F8002323706D
:101C0000504A514B10681B78C1B2002B0ED14F4C7B
:101C1000C0B223785BB2002B4FDB237824785BB211
:101C200064B21B0424021B191B1813600B1C5029DF
:101C30004ED95023464A47491078DBB2FF2202288A
:101C40004BD10868444C454D267890432A789642FB
:101C500054D9227824782E78023B5D10A31B6B4365
:101C60005201D31A10335B111843086002F054F983
:101C7000031F012B45D83A4B1B78002B06D0394B5C
:101C80001B78002B02D0002002F05EF9A122364B17
:101C900092009978354B4A431B689B188322920027
:101CA0009B181B78033B012B03D8AF20400001F0A9
:101CB00093FF01222E4BDA8270BD237824785BB229
:101CC00064B2FF33FF341B0424021B190138ABE755
:101CD000CAB2022AAED20223ACE70868254C264DD0
:101CE000267890432A78964208D9227824782D784D
:101CF000023B5B10641B63435201B2E72378DBB203
:101D0000B2E70228D5D11D4B1B78013B022B03D92A
:101D10001B4B1B78022BCCD16C20C8E79809FF1F06
:101D2000FC0FFF1F2464FF1FFF3F0000141003403F
:101D30002864FF1F0C10034000100340D50BFF1F49
:101D40007211FF1FB40003408C09FF1F680AFF1FB8
:101D5000490AFF1F94000340460AFF1F470AFF1F5E
:101D6000F908FF1F2209FF1F300DFF1F3409FF1F55
:101D7000BC0BFF1F440AFF1F450AFF1F1C09FF1F62
:101D80002309FF1F10B502F0B7F80022014B1A809B
:101D900010BDC0462064FF1F10B502F055F8A12108
:101DA000054A89009478054A61431268044B521829
:101DB000528C1A8010BDC046300DFF1F3409FF1F22
:101DC0002064FF1F10B50D4B0D4A9978A1239B008D
:101DD0004B431268D218531DD97F0A4B1B88994276
:101DE00009D2441C07D0C82805D0D2695B1A5A43CF
:101DF000054B5343C01801F0E7FF10BD300DFF1F26
:101E00003409FF1F2064FF1F7102000070B5244DCC
:101E10002B68002B28D001F017FF2B68D8402B68C7
:101E20000400002B27D002F0B7F82B68D8401D4BD8
:101E30001D4A9978A1239B004B431268D118D25CAC
:101E400091239B00002A20D0CA580132CA50174B58
:101E500017491B680868834214D3D23B181A012A19
:101E60001AD0144B186070BD01F0EEFE124B1968C9
:101E700001F082FED3E702F08FF80F4B196801F0F2
:101E80007BFED4E70D495B18E8E7CA500C4B1B6892
:101E9000DB68E418201AE4E7F530FF30E1E7C046DC
:101EA0001C08FF1F300DFF1F3409FF1F9C09FF1F77
:101EB0002464FF1FA009FF1F1808FF1F2DFF3F000C
:101EC0002C64FF1F70B504000D00282916D10300F3
:101ED000A433C2881B889B1A0B4A9BB293420DD92C
:101EE00006006A3605223100653001F0F5FF002852
:101EF00004D13100200002F01FF870BD290020003D
:101F000001F00AFFF9E7C046FE7F0000F8B50500C2
:101F1000012001F0B1FF134CA36AA26A9342FBD1E6
:101F2000114E336001F038FE10490300086010487C
:101F3000426894460F4A17680022BC4501D24268A5
:101F4000BA1A0D4802603268AD18A422E562606AD0
:101F5000520302436262094A1278002A01D00F3B01
:101F60000B60F8BD00F00040340AFF1FE408FF1FBB
:101F700028100040180AFF1F1C0AFF1F1C09FF1F22
:101F800070B580241025E405A3682B43A36001F0FD
:101F90000BFEA368AB43A36070BD0000F7B516004D
:101FA00080221C001023D2050191916805000B438B
:101FB000936000225A4BD7301A6001F055FE9D23E2
:101FC0002A002F009B00EB58CA3201210092FC37F7
:101FD000002B01D00021009A386801F0D5FE2900BD
:101FE000009BCB311A784F4BD3351A604B780A7867
:101FF0001B0213438A7812041A43CB781B0613433F
:10200000494A1BBA13604B790A791B0213438A7938
:1020100012041A43CB7931001B061343434A1BBAFF
:1020200013606B782A781B021343AA7812041A43B0
:10203000EB781B0613433E4A1BBA1360019A330226
:1020400013433C4A13603C4B22001B1B9C46032954
:102050003DDCB3089A0013005142B21A032A46D15C
:10206000354AE018511A827840781204000202437F
:10207000E05C043302430A600022FF2B4BDDF022B8
:102080002E4B12011A600F222D4B1A602D4A136835
:10209000002BFCD00023224A27491360091B321D64
:1020A0000B191B68043A180A23706070180C1B0E79
:1020B000A070E3700434002AF2DC802210213B6817
:1020C000D20501333B6093688B439360F7BD634651
:1020D000D578981893782D061B042B43157804396E
:1020E0002B43557804322D022B430360AFE7022ABD
:1020F0000AD1114AE05C511AE218527812020243E6
:102100000A6004339BB2B7E7012AB5D10A4A521AD2
:10211000E15C1160F5E7084959180A600433ACE73F
:10212000000004403C0004403800044034000440F7
:10213000300004400C00044000010440040004404E
:102140001000044014000440F7B5150080221C0064
:102150001023D2050091916807000B439360002380
:10216000654AD730136001F07FFD9D233E009B0040
:10217000F9583B00CA363200FC33002900D07FE01A
:10218000586801F001FE390032785C4BCB311A609F
:102190004B780A781B0213438A78AC4612041A4320
:1021A000CB78281D1B061343554A1BBA13604B7985
:1021B0000A791B0213438A7912041A43CB791B064E
:1021C0001343504A1BBA13604B7A0A7A1B0213431B
:1021D0008A7A12041A43CB7A21001B0613434A4A17
:1021E0001BBA1360009A2B021343484A1360220063
:1021F000474B1B1B0093009BCE785B1801938B7899
:1022000036061B0433430E78043833434E780431CA
:1022100036023343019E33600328ECDC0321A80817
:10222000431C9B002940800003292BD13849E51825
:102230005E18A9786D78E35C09042D0229431943DF
:102240003160030008330021FF2B2DDD314B324973
:1022500019600F21314B1960012327490B60304B66
:1022600019680029FCD006211B680B40042B20D0E4
:1022700080220020D20593680A318B439360FEBD13
:1022800001217DE7022908D121495D18E11849782B
:10229000E35C090219432960D3E70129D3D11C4922
:1022A0005918E35C0B60CCE7194818180160043337
:1022B000CAE7002310490B606346002B0CDC3B008F
:1022C000FC335A68102101325A608022D20593688B
:1022D00001208B439360D2E7009B9B181B68190A6F
:1022E00013705170190C1B0ED37004235B42917054
:1022F0009C440432E0E7C046000004403C00044037
:102300003800044034000440300004400C00044015
:102310000001044004000440080F000010000440C5
:102320001400044070B5061E19D002225A4B9B7946
:102330009343012B13D1594B1A78FF2A0FD15A78A6
:10234000FF2A0CD19A78FF2A09D1DA78FF2A06D120
:102350001A79FF2A03D15B79FF2B00D199E0504B0A
:102360000C201A78012A08D000224E4D1A702978C4
:102370000B00093B042B01D8212070BD4B1F012B02
:10238000FAD9454CA37B042B00D982E0A279032A19
:1023900000D97EE09A1ED2B2012A02D860881F2896
:1023A00077D9002E56D0012E73D1A0880128E3D012
:1023B000002907D1581E032803D801F0B7FB1217D4
:1023C00015122E702978481E032811D80025364B87
:1023D0001D602823237501F0A7FDA84227D0A58002
:1023E000CAE702212970EDE70421FBE70321F9E7A1
:1023F00007390129C0D82D490968C96A8906BBD5A2
:102400002B4908780028B7D1012A01D9002BB3D174
:1024100002230B708021274D2633890128782375EC
:1024200001F0A2FD80212878890101F0F5FC01234B
:10243000A380214B1B78002B0AD0FA2280211F4B4E
:1024400092001B8809025A431A4B187801F084FD48
:10245000002092E701F090FD2B78A680073B012B2E
:1024600003D917482E7001F0FFFC114B114C1A785C
:10247000002A06D080210022207889011A7001F0FC
:1024800073FD01F031FC80212078090201F06CFD20
:10249000DEE7122071E7C046A60BFF1F6B09FF1F86
:1024A0001A09FF1F1C09FF1F4809FF1F2C64FF1F8B
:1024B0002309FF1F1B09FF1F2109FF1F2C09FF1FF5
:1024C0000010004010B5002901D001F0F5FC10BD4E
:1024D000F7B5604B01919978A1239B004B435E4A6D
:1024E000060014681022E418D6235B00E058362357
:1024F000FF33E35C00279343222B41D1574B0F3A24
:102500001A600760012501F0FFFC019B1880E82399
:102510005B00E35C002B01D0B34258DD0023504F39
:10252000FB70AD33FF33E3581A68002A03D09B8851
:10253000DB439B071DD03823FF33E35C002B18D00F
:102540009B235B00E35C002B13D1D133FF33E35CAF
:10255000B3420EDAA4235B00E15AE018090A023103
:1025600001F0C2FC23000122FE33013E01351A872F
:10257000FA70E8235B00E35C002B2AD0A8B2FEBD12
:1025800003683D00002BBED081880430090A023167
:1025900001F0AAFCD6235B00E3581F60B2E72300DA
:1025A000B133BA00FF339858013781880430090AE3
:1025B000023101F099FCE8235B00E35CBB42EEDCF6
:1025C000E822F61AED1800235200A354A6E70027CC
:1025D000F1E7200001F030FB00281FD0002E1DDDA8
:1025E0007319882647190193B600200001F0FCFA00
:1025F0005A30800020184068013581880430090A6B
:10260000023101F071FC200001F0A6FBA359013357
:10261000A351BD4202D0019B9D42E6D1114BE35C28
:10262000002BABD095239B00E35C002BA6D00E4B78
:10263000E15A0029A2D00D4AA35C994202D9013384
:10264000A3549BE700231A212000A35401F0ACFB04
:1026500094E7C046300DFF1F3409FF1F00140340EC
:10266000E010FF1F5A020000720200005E0200002C
:102670000D4970B54A6E0D4CD2038B69D20BA24244
:1026800006D80B4D0224AA4204D901F0E5FA70BD28
:1026900002246442E21815007E2425402242F4D030
:1026A000A3432B438B61F0E700F000400A200000B9
:1026B000FC1C0000F8B51D4B1D4F1A78002A10D1E4
:1026C000BA7B002A02D101321A7003E0032AFAD041
:1026D000022AF8D001F028FC00220120154B1A70C4
:1026E000F8BD154B154D1C68154B9E7801232B70BA
:1026F0002878C0B200F0A2FBBB7B002B0BD101F00D
:102700005BFAA1239B007343E41883239B00E41826
:1027100023782B70E4E7032B02D101F09DFBF0E757
:102720000020022BDCD101F02FFCEAE71C09FF1F7F
:10273000A60BFF1F2309FF1F3409FF1F490AFF1FB4
:10274000300DFF1FF0B587B00EAD2F780FAD2D788F
:102750000593AC46634614000E4D0CAA12782E78F1
:1027600003930D9B009201932200059B029701F0B9
:102770004BFC2E70012C01D0042C08D1802206497C
:102780008B889343054A1278D20113438B8007B09C
:10279000F0BDC0461C09FF1F6C11FF1F7809FF1F09
:1027A0000B001B3B70B504003020E02B0DD813004C
:1027B000E025493BFF3B9BB2ED00AB4205D8034B04
:1027C000200019825A8201F057FA70BD8410FF1F51
:1027D00010B501F011FB054B00205B68052B04D9F7
:1027E000034A5268D20200D4980810BD001000407D
:1027F000FCE100E070B501F0BFFB0D4B1B68FC3342
:10280000DC691D6AFFF7E4FF6419844204D2094BB6
:1028100001241B68002B07D004220024064B1A70E9
:10282000064A93690133936101F05EFA200070BD9E
:102830002C64FF1F9809FF1F2309FF1FFC0FFF1FB8
:1028400070B50C4D2B68FC335C6A01F095FBFFF70B
:10285000BFFF2B680025FC339B6AE318834204D238
:10286000054B1B68AB4200D1051B01F03DFA280067
:1028700070BDC0462C64FF1F9809FF1FD722044B70
:1028800092009B5810B5002B00D0984710BDC04651
:102890000000FF1F10B501F0D3F8FFF7EFFF274945
:1028A000274BCA6D274C1A4084235B001343CB652A
:1028B000254B1B68186A01F0DFFA244B244A1A6082
:1028C000244B254A1A60A022244B52001A60244B44
:1028D000187801F051FA2000224901F09DFB0023F5
:1028E000A3600233A360204B2049236003232048C8
:1028F000A36001F091FB10221E4BFF201A60802282
:1029000052031A60802292031A60802212041A6015
:1029100001F01AFB012001F03FFAFA20400001F01B
:1029200063FA582001F058F9134801F045FA0120E4
:1029300001F072F9072001F04FFA10BD00F00040DD
:1029400000FEFEFF141000402C64FF1F0000034037
:102950000180063DBC00034034080000A400034091
:102960004A0AFF1F71020000C3090000FFFF3F0079
:102970002810004000E100E030750000674E336829
:1029800088331B6883F3088801F0E6F8644A6549D8
:10299000136800200B401360634B644A1B6893422A
:1029A00000D1A6E001F070FA0221614A13688B435E
:1029B0001360FFF76FFF5F4B5F4C1878C0B201F0F8
:1029C00073FA0023A3600233A3605C4B01202360F1
:1029D00001F052FA0323A36001F016FA040001F09B
:1029E0000BFA050001F010FA554B186001F0E4FAFB
:1029F000544B1968621A531EA14200D21300802260
:102A0000D203934201D39B029B0A3268D16AC90761
:102A100000D471E04C491C0C09689BB24C435943EB
:102A20002402090A641803264849FC3293680A689C
:102A300047489B1A474A0768126847499B18474A04
:102A40009A1833409208DB190A600360042B03D9FB
:102A5000013233400A6003600E684149A619300014
:102A600001F08AF83F4F3E493B68C3183B60300095
:102A7000019301F011F93C4E306808183849306074
:102A8000884205D9019B01333B6001F005F93160B3
:102A900001F00AF9354B1B78002B0DD001F0ACF991
:102AA000334B621B196812188A4232D24919091B2A
:102AB000091A304801F0B0FA2F4E337A002B0ED0AD
:102AC00001F09AF9621BF1681218914224D9491950
:102AD000091B091A294801F09FFA00233372284B79
:102AE00083F3088801F090F8002001F0CDF901F09F
:102AF000ABFA01F0C9F95CE7DC0199000234641A11
:102B00005900641A09214B438033CB40A408E418D0
:102B100089E7FA218900CCE71A49DBE72C64FF1F1B
:102B20001CF00040FFFFC1FF0C0AFF1FB64121034C
:102B300010000040490AFF1F14100040C3090000A4
:102B4000100AFF1F340AFF1F380AFF1F200AFF1F49
:102B5000280AFF1F1C0AFF1F240AFF1FC4090000C8
:102B6000710200006008FF1F2C0AFF1F1C09FF1FD5
:102B7000E408FF1F00100040740BFF1F3C100040D2
:102B800000000020DC050000A022054B92009B58AD
:102B900010B5002B01D0984710BD01F045F8FBE7B8
:102BA0000000FF1FA122054B92009B5810B5002B7F
:102BB00001D0984710BD01F037F8FBE70000FF1F78
:102BC000A222054B92009B5810B5002B01D09847CC
:102BD00010BD01F029F8FBE70000FF1FA322054B01
:102BE00092009B5810B5002B01D0984710BD01F002
:102BF0001BF8FBE70000FF1FA422054B92009B5827
:102C000010B5002B01D0984710BD01F00DF8FBE77F
:102C10000000FF1F70B501F0EFF84F4B186001F096
:102C2000E3F90400C30702D401F06EF870BD00227E
:102C30004A4B1A604A4B18780138042829D800F00A
:102C400075FF0320181C2400200001F0ADF90128B5
:102C5000ECD0444C2378042B6ED100F095FF002873
:102C6000E4D001F0E1F9582000F0B6FF0223237010
:102C7000DCE7200001F008F8E9E7200001F0ACF9FA
:102C8000E5E7200001F038F8E1E7200000F09CFFC4
:102C9000DDE701F041F90500012808D1324B1B782E
:102CA000053B012B03D82000FFF76EFFD1E72D4B2A
:102CB0001B78022B01D0052B20D1022D28D12B4BC4
:102CC0009B7BAB431CD12000FFF76CFF264B187891
:102CD0000128BED16405BCD4244925224B7B034284
:102CE00005D1233A13405A42534126331A000B7D33
:102CF0009342AED9322000F0EFFFAAE7022D07D1B0
:102D0000194B1B78052B11D12000FFF759FFDDE788
:102D1000012D0BD1012B03D12000FFF75FFF98E7B6
:102D2000062B03D12000FFF767FF92E7200000F099
:102D30007BFF022D8DD1C9E7032B04D10C4B987C6E
:102D400000F0BAFF72E7072B00D06FE7094B987BC2
:102D500000F0F2FF6AE7C0469C09FF1F9809FF1FB9
:102D60009009FF1F2309FF1F1C09FF1FA60BFF1F50
:102D7000BC0BFF1FD40BFF1FFA210A4B0A4A490064
:102D80001A640A4A5A500A4A04395A50094A083100
:102D90009A64094A5A50094A5C315A50084ADA661C
:102DA0007047C0460000FF1F4527FF1F4128FF1F37
:102DB000F527FF1F2523FF1FB526FF1FC51DFF1F7A
:102DC000991DFF1F10B500F099FE10BDF7B50B0C53
:102DD000FF270122009300233C001E001D009446A3
:102DE000019089B262469A40100008401841361896
:102DF000B6B2FF2F02D1012E00D19FB2009802403F
:102E00001A41AD18ADB2FF2C02D1012D00D19CB2F8
:102E10000133102BE6D10320012E07D1012D04D15F
:102E2000019B2401E4191C700138FEBD102EFCD159
:102E30000238102DF9D00230F7E700008023F7B5F3
:102E40009C46264B264F01932649274A274D284C5E
:102E5000284B02281AD1604638600868264E304058
:102E6000802636033043086001990978002909D18A
:102E70001660224A2A60224A2260E02219689143A1
:102E8000A03A1BE08021C9021160F2E766463E606D
:102E90000F68194E3E408027FF023E430E600199A5
:102EA000097800290DD1176001280ED1154A2A6032
:102EB000154A2260E02219689143C03A0A431A6019
:102EC000F7BD802189021160EEE7E0210F4A02433D
:102ED0002A600F4A22601A688A43F0E74B0AFF1FF4
:102EE000E0000340D800034090000340000003408E
:102EF0005000034040000340FFFFE3FF0280063D17
:102F0000804508220180063D8066082200800698E0
:102F100080550822F8B51E4B80261A680020140040
:102F20003440324232D11A681A4F32431A600122B9
:102F30003B68063093433B6000F09EFF0122164D34
:102F40002B681E432E603B680A2613433B60802794
:102F5000BF00124B1B683B4211D1013EF6B2FF2E5F
:102F600009D17E220E4B1C682B68E40B144093435E
:102F700023432B6005E0082000F07EFFE9E7002EE8
:102F8000EFD180222B68600893432B60F8BDC046C8
:102F9000C4F000405CF0004018F0004068F00040D1
:102FA00060F0004010B500F027FE01215820034AD0
:102FB00000F0DAFDFFF7AEFF10BDC046600AFF1F4C
:102FC00010B578220021034800F07EFE01F014F8CD
:102FD000002010BD3467FF1F70B5040000F0CCFF67
:102FE00000230C200B4A010059438D18515C002925
:102FF0000DD0A14208D1012300246B7000F064FFC2
:1030000000F072FE200070BD01330A2BEBD11224B8
:10301000F6E7C0463467FF1F70B5040000F0ACFF50
:10302000002319001D000D4A1078002806D0A04288
:103030000CD1557001310C320A29F5D1002B0AD17F
:1030400000F0DAFF00F050FE002070BD5078461E00
:10305000B0411B18EEE700F037FFF3E73467FF1FBE
:10306000F7B504000C20002384460E4D01926746FC
:103070005F43E85D7E19A04212D000280BD10A4BB5
:103080009C4662461B7808331370019B70707C5518
:103090007160B360FEBD01330A2BE8D10320F9E76C
:1030A0000720F7E73467FF1F3067FF1F8020F8B560
:1030B000484BC0051B68C1248360474BFF251A6835
:1030C000012313434361454BA4001A68444B40213C
:1030D0001A60444B1A68444B1A60444B1A59AA436D
:1030E0001A51C52292009E58AE4331438026995012
:1030F0009F583F49F6010F403E439E509E588027FF
:103100003602360A3043985080201A5900020A408D
:1031100002431A5104341A59364E3F043240802675
:103120003A431A511A5936061202120A32431A51F8
:1031300008341A5980260A4002431A51C3229200C9
:103140009F58B446AF4337439F509F58294E0F4076
:1031500007439F509F5837408026360437438026C8
:103160009F509F5836063F023F0A37439F50C02268
:103170001F59AF433A431A511A591202120A164301
:10318000C6221E5192009C58AC4365462C439C506D
:103190009C5800250C4020439850C72080001A58A6
:1031A000154C1140C02212020A431A50134B1B78CF
:1031B000DB08AB4201DC0020F8BD2378002B06D0F1
:1031C000A368002B00D0984701350C34EEE712209D
:1031D000F2E7C0465843FF1F5443FF1FB0F00040C2
:1031E0002C67FF1FB4F000402867FF1F00E100E0DC
:1031F000FF00FFFFFFFF00FF3467FF1F3067FF1F67
:10320000030010B51F2809D8072200201340072407
:1032100004490A78A24313430B7010BD0023062013
:10322000F5E7C0463067FF1F054B06491B780A6863
:1032300005485B0702401B0B134300200B607047DF
:103240003067FF1F1CF00040FFFFC1FF70B50C2569
:10325000FFF7EAFF0A4B1C780A4BE4086543ED18B8
:10326000002C01D1200070BD2B78002B06D06B689C
:10327000002B00D09847013C0C3DF1E71220F2E70B
:103280003067FF1F2867FF1F1FB5002102220B00B8
:1032900001910091052000F0CFFE02230B490A683E
:1032A0001A42FCD120230393039B5A1E0392002B46
:1032B000FAD1074A1368002BFCDA0B246C44200077
:1032C000012100F0B9FD207804B010BD90C8004085
:1032D00000C8004013B504000A4B0193019B002B6A
:1032E00001D1112016BDFFF7CFFF23000340044298
:1032F00005D0052000F0C0FD019B013BEDE7180063
:10330000F0E7C046FFFFFF0707B500F035FE80225B
:103310000821D205936A0191002B01D107399162EE
:1033200002210C4A11600199481E01900029FAD12E
:1033300003311160053101910199481E0190002966
:10334000FAD11160002B02D18022D205936200F0E5
:10335000CBFC07BD00C00040F0B52D4C89B02378F0
:10336000002B4FD1FEF7CEFA02232A4F03903A6882
:103370001A42FCD120230693069B5A1E0692002B6C
:10338000FAD1254E3368002BFCDA0120FFF7A2FFAB
:10339000011E02D0112009B0F0BD030003220190EC
:1033A000009005AD9F2000F047FE0321280000F0AB
:1033B00043FD02233A681A42FCD120230793079B5E
:1033C0005A1E0792002BFAD13368002BFCDA012039
:1033D000FFF780FF0028DDD10398FEF7A7FAAA784F
:1033E0006B7811041B020B4329780B4363601300B5
:1033F000113B0A49052B07D801239340A3600B60BA
:10340000012323700020C6E780231B03F6E7C04694
:103410004043FF1F90C8004000C800409808FF1FAD
:103420001E4B30B55A6818781D4B85B0D3185942D9
:103430004B4101210093002300F0C6FD194B1A4AAD
:1034400002259A6300221A6510325A658022C4212F
:103450009D65164B1648D202DA6789004258154B13
:1034600080241A4080231B041343435064234120CB
:103470000393E40500F006FA402000F003FA6562C9
:10348000039D6B1E0393002DFAD103236362FFF7A4
:103490003BFFA562FFF760FF05B030BD4C43FF1F47
:1034A00095FFFEF700C80040050001FF04E100E0C1
:1034B00000E100E0FFFF00FFF0B585B00700FEF778
:1034C00021FA022305002D4C22681A42FCD1202348
:1034D0000093009B5A1E0092002BFAD1284E3368AD
:1034E000002BFCDA0120FFF7F5FE002803D01124A1
:1034F000200005B0F0BD234B2360022322681A424E
:10350000FCD120230193019B5A1E0192002BFAD17A
:103510003368002BFCDA0120FFF7DCFE0028E6D13F
:10352000194B1F60022322681A42FCD12023029308
:10353000029B5A1E0292002BFAD13368002BFCDA50
:103540000120FFF7C7FE0028D1D1104B23600223D2
:1035500022681A42FCD120230393039B5A1E039234
:10356000002BFAD13368002BFCDA0120FFF7B2FE02
:10357000041EBCD12800FEF7D9F9B9E790C8004075
:1035800000C8004001000006A8C8004001800001FA
:1035900010B50020FFF790FF10BD000010B5064BDE
:1035A00018705960FFF73CFF00211320034AFFF712
:1035B00057FD002010BDC0464C43FF1F2134FF1FA4
:1035C000F0B5040085B003920291FEF79BF98822C2
:1035D00063035B0B52051A438023DB059D6A80233E
:1035E000274F0092BA68002601901B039A420CD91B
:1035F000F82326001B041E401C4206D08022214BCB
:1036000052025E6219680A431A60002D0BD100F065
:10361000B3FC02221C4B1A608023DB055A62013A7C
:103620009A6200F061FB0023039A934220D1002D9F
:103630000AD100F0A1FC144B03221D608023DB059E
:103640005A629D6200F050FB8023BA681B039A42C5
:1036500008D9002E06D000220A4B0C495A621A687B
:103660000A401A600198FEF761F9002005B0F0BD2C
:10367000009A0299D2181278CA540133D4E7C0468E
:103680004043FF1F00C8004000C00040FFFFFEFF96
:10369000F0B587B0029103920400FEF733F9019070
:1036A00000F06AFC802302250122234EDB053560F1
:1036B0005D629A6200F018FB204F3B682B42FCD100
:1036C00020230493049B5A1E0492002BFAD11C4D14
:1036D0002B68002BFCDA0120FFF7FCFD002802D04C
:1036E000112007B0F0BD2000039A029900F0D4FB2E
:1036F000022304003A681A42FCD120230593059B5B
:103700005A1E0592002BFAD12B68002BFCDA0120FF
:10371000FFF7E0FD051EE3D100F02EFC802303221D
:10372000DB0535605A629D6200F0DEFA0198FEF713
:10373000FDF8E0B2D5E7C04600C0004090C80040A8
:1037400000C80040F0B5802489B00600FEF7DAF822
:10375000E405A36A02250393029000F00DFC012307
:10376000304F3D606562A36200F0BEFA2E4C2368C4
:103770002B42FCD120230593059B5A1E0592002B5A
:10378000FAD12A4D2B68002BFCDA0120FFF7A2FDAD
:10379000002803D01124200009B0F0BD244B236081
:1037A000022322681A42FCD120230693069B5A1E4C
:1037B0000692002BFAD12B68002BFCDA0120FFF7D0
:1037C00089FD021EE6D11B4B03211E600300019000
:1037D0000090202000F030FC022322681A42FCD125
:1037E00020230793079B5A1E0792002BFAD12B68C0
:1037F000002BFCDA0320FFF76DFD041ECAD100F098
:10380000BBFB80230322DB053C605A629C6200F014
:103810006BFA039B002B01D1FFF776FD0298FEF7B0
:1038200085F8B8E700C0004090C8004000C80040DC
:103830000100000694C8004007B50002019104226F
:10384000000A01A9FFF724FF0EBD000073B50500B3
:1038500005240B4AA3005B429B1819686B46DE1DCA
:103860003000FFF7B3FA022804D133782B55013C1E
:10387000EFD276BD052CFCD00128FAD10230F8E752
:10388000140900111F2807D8012380228340D20584
:1038900091680B43936070473F2808D8012380222A
:1038A00020388340D20551690B435361F3E75F2809
:1038B000F1D80123802240388340D205116A0B439E
:1038C0001362E8E71F2807D8012280218240C9053A
:1038D0008B6893438B6070473F2808D80122802172
:1038E00020388240C9054B6993434B61F3E75F2859
:1038F000F1D80122802140388240C9050B6A9343E8
:103900000B62E8E71F2810D880230200DB05153A78
:103910001968012A06D820229143196019680A43C0
:103920001A60704701228240F6E73F2811D88023B1
:103930000200DB05353AD968032A06D810229143E4
:10394000D960D9680A43DA60EBE701222038824067
:10395000F5E75F28E5D842238022181A413B8340CF
:10396000D205516A99435162516A0B435362D8E7B9
:1039700010B50400012813D1A022184992050B6844
:103980005B015B0913430B60154B164A1968114024
:10399000154A0A431A60402219680A431A6010BD8A
:1039A0000028FCD101000A2000F056FB21000B206A
:1039B00000F052FBC0220A4B920019680A434021D2
:1039C0001A601A688A431A60B022044912060B680A
:1039D0005B015B0913430B60E1E7C04614F0004054
:1039E0001CF000407F00FEFF80FD010072B6074A18
:1039F0001368013313600422054B1A600023054A43
:103A000013608022D2055360FEE7C0467808FF1F8E
:103A1000C0F00040C4F0004005490B68002B05D100
:103A2000044A0A6004490A60044A13607047C046A9
:103A3000140AFF1F841E0000380AFF1FC4F0004054
:103A40000023034A1360034A1360034A136070475C
:103A500054F0004040F1004044F10040002310B514
:103A6000184C8AB0009301932378012B27D0694624
:103A7000012000F0D9F9002817D1009B12490293C8
:103A8000019B06AA0393114B02A81B680493104BD9
:103A90001B68059300F088F810220E4906A800F074
:103AA0001BFA002804D1FF23237000200AB010BDA8
:103AB0000123094A074902A8237000F075F8012084
:103AC000F4E7C0463064FF1F1029001108290011D7
:103AD0000C290011202900113464FF1F13B50124A3
:103AE0006946012000F0A0F9034B00940193FFF711
:103AF000B5FF200016BDC046BB0B000010B5FFF798
:103B00009FFFFFF7EBFF002802D0024B984710BD44
:103B1000FEE7C046E1A2000002B471464908490030
:103B2000095649008E4402BC7047C04602B4714633
:103B300049084900095C49008E4402BC7047C046F0
:103B400003B47146490840004900095A49008E44AF
:103B500003BC70470000000001B40248844601BC69
:103B6000604700BFC9A9000001B40248844601BCF7
:103B7000604700BF0167010001B40248844601BCF0
:103B8000604700BF090E000001B40248844601BC32
:103B9000604700BF01D7000001B40248844601BC61
:103BA000604700BFBD5C010001B40248844601BC0F
:103BB000604700BFDD3F000001B40248844601BCFD
:103BC000604700BFE9F6000001B40248844601BC2A
:103BD000604700BFF935010001B40248844601BCCA
:103BE000604700BF7912010001B40248844601BC5D
:103BF000604700BFD9B0000001B40248844601BC50
:103C0000604700BFED68010001B40248844601BC72
:103C1000604700BF7997000001B40248844601BCA8
:103C2000604700BFE512010001B40248844601BCB0
:103C3000604700BFE917010001B40248844601BC97
:103C4000604700BF71B0000001B40248844601BC67
:103C5000604700BFE90B010001B40248844601BC83
:103C6000604700BFD1AE000001B40248844601BCE9
:103C7000604700BF8944000001B40248844601BC8B
:103C8000604700BF116E000001B40248844601BCC9
:103C9000604700BF0934010001B40248844601BCFA
:103CA000604700BF090E000001B40248844601BC11
:103CB000604700BFD544010001B40248844601BCFE
:103CC000604700BF4DF9000001B40248844601BCC2
:103CD000604700BFB70E000001B40248844601BC33
:103CE000604700BF6137010001B40248844601BC4F
:103CF000604700BF9DA9000001B40248844601BC92
:103D0000604700BFF535010001B40248844601BC9C
:103D1000604700BFDD0A010001B40248844601BCCF
:103D2000604700BF51B8000001B40248844601BC9E
:103D3000604700BF05B2001101B40248844601BCCF
:103D4000604700BFC1F7000001B40248844601BCCF
:103D5000604700BFE94C010001B40248844601BC41
:103D6000604700BF5976010001B40248844601BC97
:103D7000604700BFE927000001B40248844601BC47
:103D8000604700BFEDA5000001B40248844601BCB5
:103D9000604700BF2144000001B40248844601BCD2
:103DA000604700BF6911010001B40248844601BCAC
:103DB000604700BF53B9000001B40248844601BC0B
:103DC000604700BF8D11010001B40248844601BC68
:103DD000604700BF8937010001B40248844601BC36
:103DE000604700BFF90D010001B40248844601BCE0
:103DF000604700BF8512010001B40248844601BC3F
:103E0000604700BFC95C010001B40248844601BCA0
:103E1000604700BF156B010001B40248844601BC35
:103E2000604700BF0D52010001B40248844601BC46
:103E3000604700BFE1AC000001B40248844601BC09
:103E4000604700BF3D71010001B40248844601BCD7
:103E5000604700BFF9ED000001B40248844601BC90
:103E6000604700BF75F8000001B40248844601BCF9
:103E7000604700BFC1A5000001B40248844601BCF0
:103E8000604700BF0189000001B40248844601BCBC
:103E9000604700BF016C010001B40248844601BCC8
:103EA000604700BF9573010001B40248844601BC1D
:103EB000604700BF8914010001B40248844601BC78
:103EC000604700BFE9D4000001B40248844601BC49
:103ED000604700BF21A9000001B40248844601BC2C
:103EE000604700BFCD4C010001B40248844601BCCC
:103EF000604700BFC115010001B40248844601BCFF
:103F0000604700BF8D82000001B40248844601BCB6
:103F1000604700BFCD0C010001B40248844601BCDB
:103F2000604700BFDD0C010001B40248844601BCBB
:103F3000604700BFA9D8000001B40248844601BC14
:103F4000604700BF85C1000001B40248844601BC3F
:103F5000604700BFED6B010001B40248844601BC1C
:103F6000604700BF8B52010001B40248844601BC87
:103F7000604700BFB352010001B40248844601BC4F
:103F8000604700BF75A9000001B40248844601BC27
:103F9000604700BF19FA000001B40248844601BC22
:103FA000604700BF6D0B010001B40248844601BCAC
:103FB000604700BF0134010001B40248844601BCDF
:103FC000604700BFC166010001B40248844601BCDD
:103FD000604700BFC56D010001B40248844601BCC2
:103FE000604700BF0534010001B40248844601BCAB
:103FF000604700BFBD0B010001B40248844601BC0C
:10400000604700BFADAE000001B40248844601BC69
:10401000604700BF9D6A000001B40248844601BCAD
:10402000604700BF2D6C010001B40248844601BC0A
:10403000604700BF6DF6000001B40248844601BC31
:10404000604700BF496D010001B40248844601BCCD
:10405000604700BF8552010001B40248844601BC9C
:08406000604700BF5D9E0011E6
:10406800020000008ABA001101000000B8B800116F
:104078000200000086BA001101000000A840FF1FDE
:1040880002000000C0B8001101000000B061FF1F6D
:104098000200000084BA0011030000002461FF1F21
:1040A80012000000020000008ABA0011010000009E
:1040B80000B900110200000086BA001101000000DA
:1040C800FDB80011020000000AB900110300000049
:1040D8005F61FF1F0200000084BA001103000000A6
:1040E8007461FF1F0200000086BA00110100000081
:1040F800FCB800110200000008B90011030000001C
:104108003561FF1F0200000084BA0011030000009F
:104118005661FF1F020000008ABA0011010000006A
:1041280044B900110200000086BA00110100000025
:10413800F141FF1F0200000056B900110100000004
:104148003BB900110200000086BA0011010000000E
:10415800F041FF1F0200000054B9001101000000E7
:104168007C61FF1F0200000086BA001101000000F8
:10417800EF41FF1F0200000052B9001101000000CA
:104188002BB900110200000086BA001101000000DE
:10419800EE41FF1F0200000050B9001101000000AD
:1041A80026B900110200000086BA001101000000C3
:1041B800ED41FF1F020000004EB900110100000090
:1041C80021B900110200000086BA001101000000A8
:1041D800EC41FF1F020000004CB900110100000073
:1041E8001CB90011020202020202000000000000D5
:1041F80016150000214B0011E54A001198B900116D
:1042080090011D0018001800FFFF070102030405B4
:104218000602010600000000000000000000000087
:104228000000000000000000000000000000000086
:1042380003000000020000008ABA0011010000001B
:10424800B8B900110200000086BA00110100000090
:10425800AC42FF1F02000000C2B9001101000000BB
:10426800AA61FF1F0200000084BA001103000000C9
:104278001464FF1F0200000086BA0011010000004C
:10428800AC42FF1F02000000C0B90011010000008D
:10429800AC61FF1F0200000084BA00110300000097
:1042A8000C64FF1F12000000000100000000011153
:1042B800FFFF0000504859360000000000000000D1
:1042C8000B000500F0000000B400002800280028BA
:1042D8003075A000A000A000A00000080008E001C0
:1042E800F000100010001000100010001000500026
:1042F8005000500010001000D0070000000000001F
:104308000F0001000500307507001000010081FF53
:1043180000000000FF000000457000114D6E001104
:10432800DD6B0011FFFF0100FF000000619A001122
:10433800DD970011F5960011000000000000000054
:1043480000000800040000003B0001085902E001D9
:1043580088212800FF000000020000008ABA00112E
:104368000100000050BB00110200000086BA0011D5
:1043780001000000DD43FF1F0200000082BA0011A7
:1043880001000000EC67FF1F0200000086BA001160
:1043980001000000DC43FF1F0200000080BA00118A
:1043A80001000000DA43FF1F0200000086BA001176
:1043B80001000000D843FF1F020000007EBA001170
:1043C80001000000D043FF1F180018001D009001D5
:1043D8000200000302020000020000008ABA001175
:1043E8000100000064BB00110200000086BA001141
:1043F800010000002044FF1F020000007CBA0011E9
:1044080000000000000000000200000084BA001153
:0A441800030000000C68FF1F20FFE6
:040000051FFF184180
:00000001FF
